:020000040000FA
:100000000C94C50700000000000000000000000084
:100010000000000034C60000A6C60000000000007A
:1000200000000000000000000C941FCE0C948DC84E
:1000300000000000000000000000000000000000C0
:1000400000000000000000000000000000000000B0
:1000500000000000B5C50000000000000000000026
:10006000000000001BC5000084C500000000000067
:100070000000000000000000000000000000000080
:10008000E6C60000000000000000000000000000C4
:10009000000000000000000018FFFFFFFFFFFFFF4F
:1000A00000000000FF03000000000000000000004E
:1000B000000000000000000000000025303458005F
:1000C000253032640025303258000000080000005E
:1000D00000000000000000080000073866A81200B9
:1000E0000000292E2E47D391FF0D05C000060020E9
:1000F00028C5CA751322E534073018166C434091A1
:10010000876BF85610E92A001F4100597F3F81355F
:10011000090000F113F114F11CF120F121F122F199
:1001200023F124F125F126F127F129F12AF138F103
:1001300039F13AF13BF13CF13DF13EF140F141F151
:1001400042F143F144F145F146F147F148F149F1FB
:100150004AF14BF14CF14DF14EF14FF150F151F1AB
:1001600052F153F154F155F15AF165F166F167F12D
:1001700068F169F16AF16BF16CF1B3F1B6F1B7F1C5
:10018000B8F1C2F1C3F1DFF1E0F1E1F1E2F1E3F145
:1001900070F171F172F173F174F175F176F177F13B
:1001A00078F179F17AF17BF17CF17DF17EF17FF1EB
:1001B00080F181F182F183F184F185F186F187F19B
:1001C00088F1A0F1A1F1A4F1A5F1A6F1A7F1A8F1A0
:1001D000A9F1AAF1ACF1ADF100F401F402F403F4D9
:1001E00004F406F407F408F409F40AF40BF40CF42C
:1001F0000DF40EF40FF410F411F412F413F414F4DB
:1002000015F416F417F41BF41CF41DF41EF41FF47B
:1002100020F421F422F424F425F42CF42DF42EF40B
:1002200036F437F438F439F43AF43DF43EF43FF45C
:1002300040F441F442F443F446F447F448F449F4FA
:100240004AF44BF44CF44DF44EF44FF450F451F4A2
:1002500052F453F454F455F456F458F459F45AF44F
:100260004BF55EF45FF460F461F462F463F464F4FB
:1002700065F466F467F468F469F46AF46BF46CF49A
:100280006DF46FF470F472F474F476F478F47AF434
:100290007CF47EF471F473F475F477F479F47BF400
:1002A0007DF47FF480F481F482F483F484F485F4A3
:1002B00086F487F488F489F48AF48BF48CF48DF452
:1002C0008EF48FF490F491F493F494F495F497F4FD
:1002D00098F499F499F49CF49DF4ACF4ADF4AEF474
:1002E000B0F4B1F4B2F4B3F4B4F4B5F4B6F4B7F4D2
:1002F000B8F4B9F4BAF4BBF4BCF4BDF4BEF4BFF482
:10030000C0F4C1F4C2F4C3F4C4F4C6F4C7F4C8F42E
:10031000C9F4CAF4CBF4CCF4CDF4CEF4CFF4D0F4D9
:10032000D2F4D4F4D6F4D1F4D3F4D5F4D7F4D8F489
:1003300000F501F502F514F515F516F517F518F5A4
:1003400019F520F522F523F524F525F532F533F5D9
:1003500034F535F536F537F538F539F53AF53BF539
:100360003CF53DF53EF53FF540F541F542F543F5E9
:1003700044F545F550F551F554F55EF55FF560F53A
:1003800061F562F563F564F565F566F567F568F5A1
:1003900069F56AF56BF56CF56DF56EF503FA04FA1F
:1003A00005FA06FA07FA08FA09FA0AFA0BFA0CFA39
:1003B0000DFA0EFA0FFA10FA3FFA43FA44FA45FA28
:1003C00046FA47FA48FA49FA4AFA4BFA4CFA4DFA11
:1003D0004EFA4FFA50FA80FA86FA96FA97FA98FA95
:1003E00070F572F573F574F576F579F57AF580F5B3
:1003F00081F582F583F584F598F599F59AF59BF5E5
:100400009CF59DF59EF59FF5A0F5A1F5A2F5A3F548
:10041000A4F5A8F5A9F5AAF5ABF5ACF5ADF5AEF5E3
:10042000AFF5B2F500F630F670F611FF48FF67FF42
:10043000E0F4E1F4E4F4E7F4E8F4E9F4EAF4EBF4EA
:10044000ECF4EDF4EEF4F0F4F0F4F6F4F7F400006C
:100450000100010001000100010001000100013F55
:1004600001FF01FF01FF000800440100010001013C
:100470000154019D0100010001820182018201827B
:100480000182018201820182018201820182018254
:10049000018201820182018201820182011101B087
:1004A00001B20114017E01D801D401D601DA01DCC8
:1004B0000160017101820042012201010101014834
:1004C000011401040127012100270020018C01757E
:1004D00001C20102010C01040110017501C2013ABF
:1004E0000174012801FF0117018001000180010052
:1004F0000130017001000100011101890106012292
:1005000001800104010001000100012001C001C0BF
:10051000010101140100011C012B01300154019C57
:1005200001580111011A01970196010101FE01B163
:10053000014F010C011C01FD01800141013B01152E
:10054000012001F001C00188016801000170019ED5
:1005500001AA01010100015B01380158010401CC2D
:1005600001C4011A01090149012001D001B001F8BB
:10057000013F01FF0180010101FF01EF01030100C3
:1005800001FF01EF01C3017F01D20188014401E0B5
:1005900001C001F0017001C101000101000001343E
:1005A000018901B4018C01BA01870134018901007C
:1005B000010001000176018E013101730114014136
:1005C00001FB01FF0101010001000100010001FF29
:1005D00001FC010201FF0100010001000101010015
:1005E000010F01A6010401F9010001000100010051
:1005F000010D01C3010301D301000100010001004D
:10060000012201E8010001000100012A0138011066
:1006100001100186018601000100010101FF01FFB7
:1006200001FF01FF01FF01FF01FF01CC01CC01CC63
:1006300001CC01CC01CC01CC01FF01FF0100010084
:100640000100010001000129017F0134018901FA43
:10065000010B0195013801F9013100BC001400F6CD
:100660000004000200FC000100FF0141010601003E
:100670000104010B018B010001000104015001B2D2
:10068000010001E701D301FA0100010101D0017D60
:100690000153012F0124011F001201000102018AF0
:1006A00001BD007D0125013E0155016B0172017FF5
:1006B0000100010001410000000001F001000105FE
:1006C00001E0017D0180014701000100019401105A
:1006D0000100010001000100013701290137013348
:1006E0000131012F0139013A012901370133012F6D
:1006F0000139013A0104012101210120011F011EDC
:10070000011E011D011B01200120012001200120EB
:1007100001210101011C01000100010001B0018063
:100720000100012001000103010001580181016A5B
:1007300001110185017501000100010001C10100E5
:10074000011B01730188012C013A0107010301001B
:10075000010101000139019701FF01FF01000110B2
:10076000010001000100010001000000006C010215
:1007700001FB01870109014B0100011F011F013726
:100780000103010001000150013C04001F3F1E3F16
:100790003D1F3D3E3D1E05002F3F2E2F3D0F0E2ECF
:1007A0003D0E06002F3F2E2F0E0F0E1E3D3D070063
:1007B0003F3F3E1F0E3E0E1E3D3D08003F3F3E1F89
:1007C0000E3E0E1E3D3D09003F3F3E1F0E3E0E1EDB
:1007D0003D3D0A003F3F3E1F1E3E0E1E3D3D0B00AD
:1007E0003F3F3E1F1E3E0E1E3D3D0C003C3E1C2E5C
:1007F0000C1E2B2D1B1D0D001D3E3C2E2C1E0C2DEA
:100800002B1D0E000E3E3D2E0D1E2C2D0C1D0F001F
:100810002E3E1E2E2D1E3C2D2C1D10003E3E1E2E4B
:100820003D1E0D2D3C1D11003E3E1E2E3D1E1D2D5C
:100830000D1D04003C2C0C2C1B2C1B1C0B3B050021
:100840000D0D0C0D1B3C1B1C0B3B06001D0D0C1D48
:100850002B3C1B1C0B3B07001D1D0C1D2B3C1B1CAC
:100860000B3B08002D1D1C1D2B3C2B0C1B3B0900BA
:100870002D1D1C1D2B3C2B0C1B3B0A003D2D1C1D54
:100880003B3C2B0C1B3B0B003D2D1C1D3B3C2B0C08
:100890001B3B0C00392939191919191909190D00AF
:1008A0002A391A0A390A2939290A0E002B3A1B1B40
:1008B0003A1B1A0B1A3A0F000C1B3B3B1B3B3A3BF3
:1008C0003A1B10000D3C2C2C2B0C0B3B0B1B11006E
:1008D0000D0D2C3C3B1C0B3B0B1B12000C0C0C0C91
:1008E0001D0C3C0C2C0C13000C0C0C0C0E0C2D0CC9
:1008F0001D0C14000C0C0C0C1E0C3D0C2D0C1500CA
:100900000C0C0C0C1E0C3D0C2D0C16000C0C0C0CC5
:100910002E0C0E0C3D0C17000C0C0C0C2E0C0E0C9F
:100920003D0C18000C0C0C0C0C0C0C0C0C0C1900D5
:100930000C0C0C0C0C0C0C0C0C0C1A000C0C0C0CF5
:100940000C0C0C0C0C0C1B000C0C0C0C0C0C0C0CE4
:100950000C0C1C000C0C0C0C0C0C0C0C0C0C1200D9
:100960000A0A0A0A1A0A3A0A2A0A13000A0A0A0A88
:100970000B0A3B0A1B0A14000A0A0A0A1B0A3B0A52
:100980002B0A15000A0A0A0A1B0A3B0A2B0A160040
:100990000A0A0A0A2B0A0C0A3B0A17000A0A0A0A60
:1009A0002B0A0C0A3B0A18000A0A0A0A0A0A0A0A4F
:1009B0000A0A19000A0A0A0A0A0A0A0A0A0A1A008C
:1009C0000A0A0A0A0A0A0A0A0A0A1B000A0A0A0A80
:1009D0000A0A0A0A0A0A1C000A0A0A0A0A0A0A0A6F
:1009E0000A0A01000F3F0E3F2D2F2D1F3D3E020032
:1009F0000F3F0E3F2D2F3D0F3D2E03001F3F1E3F8B
:100A00003D1F3D3E3D2E01000C3C0B3C2A2C2A1C78
:100A10003A3B02000C3C0B3C2A2C3A0C3A2B0300CC
:100A20001C3C1B3C3A1C3A3B3A2B00002F2E0E0E6E
:100A30003D01003E0E2D0D3C02001E1E1E3D2D03ED
:100A4000001E1E1E3D2D00002C2B0B0B3A01003BFF
:100A50000B2A0A3902001B1B1B3A2A03001B1B1B13
:100A60003A2A3F0102043F081020D00024F400C0BD
:100A7000EF0B08401FC00024F40002013031323374
:100A800034353637383941424344454630313233C4
:100A9000343536373839616263646566FA93EA93B0
:100AA000BA93AA939A938A937A936A935A934A939E
:100AB0003A932A931A920A921FB61A920024B0917E
:100AC000CE00E0911102FF27E856FC4FB083B091B1
:100AD0002B02B01519F0A02DB02D02C0A1E0B02D51
:100AE0009D01B0919803B43219F0A02DB02D02C031
:100AF000A1E0B02D2A233B232015300549F1B09108
:100B00001102B03648F4B0912B02B01529F4B0911F
:100B10001102BF5FB0931102B0911102B03629F4F7
:100B2000B0E2B093980300921102E0911102FF2706
:100B3000EA56FC4FB081BD3059F4E0911102FF2715
:100B4000E956FC4FB081BA3019F4B1E0B0932B02F2
:100B500019901FBE09901990299139914991599185
:100B60006991799189919991A991B991E991F991B5
:100B70001895FA93EA93BA931A920A921FB61A92A8
:100B80000024B0911002B01571F0B0911002B15074
:100B9000B0931002E0911002FF27E850FC4FB081A3
:100BA000B093CE0005C0B091C900BF7DB093C9001D
:100BB00019901FBE09901990B991E991F991189572
:100BC000FA93EA93BA93AA931A920A921FB61A92C8
:100BD0000024629910C0A0911C02B0911D02A031A6
:100BE000B00548F0A0911C02B0911D021197A0938E
:100BF0001C02B0931D02A0912602B091270210970B
:100C000049F0A0912602B09127021197A0932602E5
:100C1000B0932702B091D202BF5FB093D202B1E08D
:100C2000B0932C02B091D202BF77B01519F4B1E0A5
:100C3000B0933002B091D202BF77BF3719F4B1E060
:100C4000B0933102B0912D02B13081F48A98899825
:100C5000B0919402B8B9889A8898899AB091930211
:100C6000B8B9889A88988A9A00922D0219901FBE66
:100C700009901990A991B991E991F9911895FA9370
:100C8000EA93BA93AA939A938A937A936A935A931C
:100C90004A931A920A921FB61A920024B091440203
:100CA000B3FD37C0B0914402B1FF0AC0A091470222
:100CB000B09148021196A0934702B093480209C030
:100CC000A0914702B09148021197A0934702B093B8
:100CD0004802B0914402B2FF17C0A0914702B09100
:100CE0004802B095A195BF4F80914B0290914C0264
:100CF000A80FB91F0E94C322A13BB0052CF4B091EC
:100D00004402BB7FB0934402B0914602BF5FB093F0
:100D10004602A0914702B091480280914B02909107
:100D20004C02A817B90771F4B0914402B860B093AF
:100D300044020E94FB22B0914302BF7EB093430263
:100D40000E94F2220092450219901FBE099019904C
:100D5000499159916991799189919991A991B99103
:100D6000E991F9911895FA93EA93BA93AA939A9311
:100D70008A937A936A935A934A931A920A921FB665
:100D80001A920024B0914402B3FD37C0B0914402DE
:100D9000B1FF0AC0A0914902B0914A021196A093F6
:100DA0004902B0934A0209C0A0914902B0914A0297
:100DB0001197A0934902B0934A02B0914402B2FF46
:100DC00017C0A0914902B0914A02B095A195BF4FBA
:100DD00080914D0290914E02A80FB91F0E94C3222C
:100DE000A538B0052CF4B0914402BB7FB093440207
:100DF000B0914602BF5FB0934602A0914902B09104
:100E00004A0280914D0290914E02A817B90771F4E1
:100E1000B0914402B860B09344020E94FB22B091AA
:100E20004302BF7DB09343020E94F222009245022A
:100E300019901FBE09901990499159916991799122
:100E400089919991A991B991E991F9911895FA939C
:100E5000EA93BA93AA939A938A937A936A935A934A
:100E60004A931A920A921FB61A920024B091440231
:100E7000B3FD7AC0B0914502BF5FB0934502B09117
:100E80004402B2FF15C0B8E0B0934F02B0918800A1
:100E9000BF3F68F4B0918800B13F30F4B091880052
:100EA000B15FB093880003C0BFEFB093880037C034
:100EB000B0914602B43090F4B0918800BF3F68F41E
:100EC000B0918800BC3F30F4B0918800BC5FB09313
:100ED000880003C0BFEFB09388001FC0B0914602E6
:100EE000B83070F0B0914F02A0918800BA1738F472
:100EF000B0918800A0914F02BA1BB09388000DC03A
:100F0000B0918800B13148F0B0918800B53028F038
:100F1000B0918800B450B093880000924602B0911E
:100F20008800B0935002B0914502B131E0F0B09129
:100F30004402B860B09344020E94FB22B091440284
:100F4000B0FF08C0B0914302BF7DB860B068B093F5
:100F5000430207C0B0914302BF7EB460B068B09353
:100F600043020E94F22202C00092450219901FBE65
:100F70000990199049915991699179918991999123
:100F8000A991B991E991F9911895002401E00EBF5A
:100F90000FE00DBFD2E0C0E1B2E0A0E1F0E0E8E98F
:100FA00090E089E715901D920197E1F7B2E0A9E87A
:100FB00091E086ED0D920197E9F70C94130FFB2F4A
:100FC000F033F9F0F133E9F0F233D9F0F333C9F04B
:100FD000F433B9F0F533A9F0F63399F0F73389F02B
:100FE000F83379F0F93369F0F13471F0F23471F0DB
:100FF000F33471F0F43471F0F53471F0F63471F0CB
:101000000FC0AB2FAF700DC0AAE00BC0ABE009C0A2
:10101000ACE007C0ADE005C0AEE003C0AFE001C08A
:101020000000BA2F0895A0FF04C091E09093B00291
:1010300002C00092B002A1FF04C091E09093B102FF
:1010400002C00092B102A2FF04C091E09093B202EC
:1010500002C00092B202A3FF04C091E09093B302D9
:1010600002C00092B302A4FF04C091E09093B402C6
:1010700002C00092B402A5FF04C091E09093B502B3
:1010800002C00092B502A6FF04C091E09093B602A0
:1010900002C00092B602A7FF04C091E09093B7028D
:1010A00002C00092B702B0FF04C091E09093C0026A
:1010B00002C00092C002B1FF04C091E09093B90257
:1010C00002C00092B902B2FF04C091E09093BA024C
:1010D00002C00092BA02B3FF04C091E09093BB0239
:1010E00002C00092BB02B4FF04C091E09093BC0226
:1010F00002C00092BC02B5FF04C091E09093BD0213
:1011000002C00092BD02B6FF04C091E09093BF02FE
:1011100002C00092BF02B7FF04C091E09093BE02EC
:1011200008950092BE0208959091B002913009F4A2
:10113000A1609091B102913009F4A2609091B20245
:10114000913009F4A4609091B302913009F4A86041
:101150009091B402913009F4A0619091B502913060
:1011600009F4A0629091B602913009F4A0649091C4
:10117000B702913009F4A0689091C002913009F44F
:10118000B1609091B902913009F4B2609091BA02C5
:10119000913009F4B4609091BB02913009F4B860C9
:1011A0009091BC02913009F4B0619091BD029130F0
:1011B00009F4B0629091BE02913009F4B068909148
:1011C000BF02913009F4B0640895B02D0000B02D35
:1011D000A0E2EB2FFF27E850FC4FA083BF5FB036A3
:1011E000B8F30092100200000895B02D0000B02D59
:1011F000A0E2EB2FFF27E856FC4FA083BF5FB0367D
:10120000B8F3009211020000089500926900009264
:101210006A000DBA0CBA009268000BBA00926B001B
:1012200005BC07BC08BC00926E0005BA00928000A5
:101230000092900000928100009291000092820042
:101240000092920000926F000092710006BA009224
:10125000700007BA08BA0092C9000895689A0E94FF
:10126000CB220E9465220E943B300E94BF300E9428
:10127000A0300092CD00B3E3B093CC00B8E9B093B6
:10128000C900B6E0B093CA008398B0B3B760B0BBF2
:10129000BFEFB7B98A9A8898BAB1BF79BAB95D98E1
:1012A0006A986998699A719A699A719869980E947E
:1012B00065229BDF8ADFB2E0B4BDB0E8B7BDB4E021
:1012C000B5BDB2E0B0936E000895F8940895789497
:1012D00008953A932A931A9322971A2F2B2F188343
:1012E0002983000001C00000B0EA0E94AA22B130A8
:1012F000D1F3B9810E948522B8810E948522000025
:1013000001C00000B1EA0E94AA22B130D1F3B1E0DD
:101310000E9496223B2F0E94B8220000B32F2296F3
:1013200019912991399108953A932A931A93229702
:101330009D01192F0000288339837098000001C097
:101340000000B0EA0E94AA22B130D1F30000B981B6
:101350000E948522B8810E948522B12F0E94852299
:101360000E94B822709A000001C00000B1EA0E94F9
:10137000AA22B130D1F30000B1E00E9496220E946F
:10138000B8220000229619912991399108953A9333
:101390002A931A930A93FA92EA928D017C0197019B
:1013A0000000D801922FC0DF232F3327D8011196D8
:1013B000922FBADF0000E990F990099119912991D3
:1013C000399108953A932A931A930A938D01202D07
:1013D000302D0000D80111967CDF2B2F302D322FBD
:1013E0002227D80176DF2B2B0000D9010991199112
:1013F0002991399108953A932A93B1E02B2FB09116
:101400002802B13001F5302DA32FBB27A054B04FD7
:10141000E32FFF27E456FC4F908186DF3F5F3C308F
:1014200098F3302DA32FBB27A054B04F52DFE32FEA
:10143000FF27EC53FD4FB0833F5F3C3098F3699832
:101440000092280211C0302DE32FFF27E456FC4FF5
:10145000B081E32FFF27EC53FD4FA081BA1709F0AD
:10146000202D3F5F3C3080F3B22F299139910895B0
:10147000A02DEA2FFF27E856FC4F9081EFE0FF27D1
:101480007A2F8827E71BF80BEB0FF01DE850FC4F75
:101490009083AF5FA03168F39B2F905FB92F0895C1
:1014A0003A932A9323970000E0911002FF27EA5015
:1014B000FC4FB0812B2FB0911002B3503B2F07C0CF
:1014C000E32FFF27E850FC4FB0812B273150E32F4B
:1014D000FF27E850FC4FB081BA3211F0323080F76C
:1014E0000000A22FBB27BA93AA93DE0112968DE3C8
:1014F00092E00E9459312296B981B093FA03B881E3
:10150000B093FB0323962991399108953A932A9336
:101510001A93B2E03B2F0000B09199032B2F07C024
:10152000E32FFF27E856FC4FB0812B273F5FE32FC7
:10153000FF27E856FC4FB081BA3211F0303680F305
:10154000E32FFF27E656FC4FB08139DD1B2FE32F39
:10155000FF27E756FC4FB08132DDBB0FBB0FBB0F3F
:10156000BB0F1B0F21270000201511F4B1E001C0B3
:10157000B02D19912991399108953A932A931A938C
:101580000A93FA92A0E1B02D1DDF9D01293CF2E300
:101590003F0718F4A02DB02D02C0A1E0B02DFA2E07
:1015A0000B2F2832F3E23F0718F0A02DB02D02C018
:1015B000A1E0B02DFA2A0B2BF014000519F0A6E1DA
:1015C000B6E29D0120939B0230939C020000A2E1B1
:1015D000B02DF8DE9D012832F3E23F0720F0293CD0
:1015E000F2E33F0718F0A8E6B9E29D0120939D02BF
:1015F00030939E020000A4E1B02DE4DE9D0128326C
:10160000F3E23F0720F0293CF2E33F0718F0A6EE93
:10161000BDE29D0120939F023093A0020000A6E14D
:10162000B02D57DE1B2F123419F4A02DB02D02C09F
:10163000A1E0B02DFA2E0B2F143519F4A02DB02DEA
:1016400002C0A1E0B02DFA2A0B2BF014000511F016
:10165000B4E51B2F1093A1020000A7E1B02D39DEE5
:101660001B2F123411F4113411F0B2E41B2F10931C
:10167000A2020000B1E0B093A5020092A602000011
:10168000A1EEBDE026DEB093A302A0EEBDE021DE18
:10169000B093A4020000A2EFBDE01BDEB0931502E0
:1016A000B0911502BB3018F4A02DB02D02C0A1E0FE
:1016B000B02DFA2E0B2FB0911502B01519F0A02DF8
:1016C000B02D02C0A1E0B02DFA2A0B2BF0140005BA
:1016D00019F0B1E0B0931502102DA12FBB27A05433
:1016E000B04FF7DDE12FFF27EC53FD4FB0831F5FB5
:1016F0001C3098F3F9900991199129913991089525
:101700003A932A931A930A93FA92EA92DA92CA9235
:10171000BA92AA929A920B2FE92EFA2E982E0E9434
:10172000FC250E945D22B01589F4AFEFBFEF6D017B
:101730000000B1E00E944B2206C0F1E0CF1AD008B1
:10174000000000000000C014D004B9F70000A02F72
:10175000BB2795E0AA0FBB1F9A95E1F7AE0DBF1D01
:1017600031DEA0939102B09392020000A02FBB271C
:1017700095E0AA0FBB1F9A95E1F71696AE0DBF1D17
:1017800021DEA0939302B09394020000A02FBB2708
:1017900095E0AA0FBB1F9A95E1F71396AE0DBF1DFA
:1017A00011DEA0939502B09396020000A02FBB27F4
:1017B00095E0AA0FBB1F9A95E1F71296AE0DBF1DDB
:1017C00088DDB09397020000A02FBB2795E0AA0FF9
:1017D000BB1F9A95E1F71596AE0DBF1D7ADDB0934C
:1017E00098020000A02FBB2795E0AA0FBB1F9A9577
:1017F000E1F71896AE0DBF1D6CDDB09399020000A5
:10180000B8E1B0939A02B0919802B83010F000920B
:101810009802B0919702B63521F4B02D0E9439227A
:1018200003C0B1E00E9439220E94DF2900000E941B
:10183000F52A00000E94C22D00000E940B2F00001C
:10184000F1E09F1609F060C0A02CB02D0E94272265
:10185000102D202D00001F5F2F4F1835FBE12F07A3
:10186000C8F3B1E03B2F0000313019F4B1E0BB2EDA
:1018700007C0323019F4BAE0BB2E02C0B4E6BB2E6A
:101880003F5F343080F3B0EEB093D302B0EFB0934B
:10189000D402B2E7B093D502A092D602302D000058
:1018A000E32FFF27ED52FD4FB0810E943A303F5F9A
:1018B0003530A8F301C00000A4E3B0E31097D9F3DA
:1018C000102D202D00001F5F2F4F1834F1E72F0738
:1018D000C8F3302D0000E32FFF27ED52FD4FB081FC
:1018E0000E943A303F5F3530A8F301C00000A4E306
:1018F000B0E31097D9F3102D202D00001F5F2F4F5C
:10190000103BF6E32F07C8F3A0919F02B091A0020D
:101910008091910290919202A817B90720F4B1E04A
:101920000E94272203C0B02D0E942722B1E00E940E
:101930004B220E941526B1E0B0932D02000001C099
:101940000000B0912D02B130D9F39990A990B990CF
:10195000C990D990E990F9900991199129913991FB
:1019600008953A932A93BDE3B0933803B1E0B0935E
:1019700012020E944530A091D802BB27A077B02D5B
:10198000FD01F03009F06DC0E030F1F0E03109F414
:1019900068C0E03209F465C0E03309F462C0E034A5
:1019A00009F45FC0E03509F45CC0E03621F0E037AF
:1019B00009F457C056C0BAE3B0933803B1E0B0930E
:1019C00012020E9445304DC000923803BBEFB09325
:1019D0003903B2E0B09312020E944530B091D902AF
:1019E000B01559F400923803B4E3B0933903B2E070
:1019F000B09312020E94453034C0B091D9022B2F0F
:101A0000BFEFE22FFF27E85CFC4FB083B22FBF5F30
:101A1000B09312020E9445300000E7DBB091D9027A
:101A20002B2FB3E03B2F0BC0E32FFF27E852FD4FD6
:101A3000B081E32FFF27EB56FC4FB0833F5FA32F0E
:101A4000BB27822F99270296A817B9076CF3B32FEB
:101A5000B350B0931102B1E0B0932902B1E0B0935A
:101A60002B022991399108953A930E948430BDE365
:101A7000B0933803B1E0B09312020E944530A091B8
:101A8000D802BB27A077B02DFD01F030D9F4E030AB
:101A9000C9F0E031B9F0E032A9F0E03399F0E03478
:101AA00089F0E03579F0E03669F0E03709F00AC0F6
:101AB0000E948430BBE3B0933803B1E0B0931202CC
:101AC0000E944530B0911002B0931202302D0BC02D
:101AD000E32FFF27E850FC4FB081E32FFF27E85C9E
:101AE000FC4FB0833F5FB09110023B1788F3B0EC1E
:101AF000E0911202FF27E85CFC4FB083B091120224
:101B0000BF5FB0931202B0911202E0911202FF2760
:101B1000E85CFC4FB083B0911202BF5FB093120239
:101B2000BFE7E0911202FF27E85CFC4FB083B09161
:101B30001202BF5FB09312020E9445300E948430AF
:101B4000B5E3B0933803B1E0B09312020E94453080
:101B5000399108953A932A931A930A93FA92EA9242
:101B6000002D102D202D302D802D902DA02DB02D4D
:101B7000402D502DBA0160197041DB01FD01B49177
:101B80008B2F902DA02DB02DBA2FA92F982F8827FD
:101B9000BA016F5F7F407B01F701F4908F29BA2F64
:101BA000A92F982F8827BA016E5F7F407B01F7012C
:101BB000F4908F29BA2FA92F982F8827BA016D5F2B
:101BC0007F407B01F701F4908F29082719272A27E6
:101BD0003B274C5F5F4F5E3068F26CEF7FEFDB01BD
:101BE000FD01B4918B2F902DA02DB02DBA2FA92FD0
:101BF000982F88276DEF7FEF7B01F701F4908F29F5
:101C0000BA2FA92F982F88276EEF7FEF7B01F7015E
:101C1000F4908F29BA2FA92F982F88276FEF7FEF85
:101C20007B01F701F4908F29082719272A273B27E2
:101C3000001510052005300511F4B02D01C0B1E0EC
:101C4000E990F990099119912991399108953A9360
:101C50002A931A930A93FA92EA92DA92CA92BA9261
:101C6000AA929A928A92802C902CA02CB02C002DB3
:101C7000102D202D302DE02CF02CD7012ADB0B2F3E
:101C8000102D202D302D322F212F102F0027D7017E
:101C900011961FDB0B2B322F212F102F0027D7017E
:101CA000129617DB0B2B322F212F102F0027D70175
:101CB00013960FDB0B2B80269126A226B326FCEF72
:101CC000EF1AFFEFFF0AFEE0FF16B8F2ACEFBFEF2E
:101CD0006D01D601FD01B4910B2F102D202D302D5B
:101CE000322F212F102F0027ADEFBFEF6D01D6014E
:101CF000FD01B4910B2B322F212F102F0027AEEFB7
:101D0000BFEF6D01D601FD01B4910B2B322F212FB6
:101D1000102F0027AFEFBFEF6D01D601FD01B49189
:101D20000B2B80269126A226B32680149004A004B3
:101D3000B00411F4B02D01C0B1E089909990A99040
:101D4000B990C990D990E990F99009911991299188
:101D5000399108953A932A931A930A93FA92EA9240
:101D6000A1EEBDEF7D01D701FD01B4912B2F302DE8
:101D7000322F2227A0EEBDEF7D01D701FD01B491E6
:101D80002B2BA1EEBDE0A5DA0B2F102D102F002775
:101D9000A0EEBDE09EDA0B2B2017310711F4B02D19
:101DA00001C0B1E0E990F990099119912991399117
:101DB00008953A932A931A930A93FA92202D302D7C
:101DC000D901A019B0418D01D801FD01B491FB2EBC
:101DD000D9019F2DA9DAD901B02D109711F4699A74
:101DE0007198D901B02DA038B00511F4699A719A93
:101DF0002F5F3F4F303120F36998F9900991199185
:101E0000299139910895A6DEB13029F40000699A2C
:101E1000719AFCCF08959EDFB13059F218DFB130CE
:101E200009F4C7CF0895E397F894A895B4B7B77F9E
:101E3000B4BFB0916000B861B093600000926000E0
:101E400000000CDAE0DF0E94352997DBA0EBBFE051
:101E500040DAB0931402B0911402B01519F0A02D1D
:101E6000B02D02C0A1E0B02D1D01B0911402BB3015
:101E700018F4A02DB02D02C0A1E0B02D2A2A3B2AD3
:101E80002014300419F0B1E0B093140220DAB1E06C
:101E9000B09316020092BE020092BF020092C002EE
:101EA0000092C102B1E0B093B602B1E0B093BC02BF
:101EB000B1E0B093BD020092C3020000B0912B02CA
:101EC000B13009F0F8C2000021DBB13009F0ECC2FA
:101ED00092DAB13009F0E8C2B091A903B883B881B1
:101EE000FB2FF63409F451C0F93409F431C2F0354E
:101EF00049F0F33509F4A1C1F73531F1F83509F4AA
:101F000021C1D0C262D90E944C24AB2FBB27AF7332
:101F1000B02D1D0109D9A07C2A2A3B2AD10183D8E2
:101F2000B1E0B09316020092BE020092BF0200928E
:101F3000C0020092C1020092B602B1E0B093BC02AE
:101F4000B1E0B093BD02B0C240D90E944C24AB2F87
:101F5000BB27AF73B02D1D01E7D8A07C2A2A3B2AEE
:101F6000D10161D8B091B602B01509F09DC2B0910F
:101F7000B902B01509F098C2B091B702B01509F0D6
:101F800093C2B0E4B09316028FC21FD90E944C24B2
:101F9000AB2FBB27AF73B02D1D01C6D8A07C2A2A5A
:101FA0003B2AD10140D8B091B602B01509F07CC2ED
:101FB000B091B902B01509F077C2B091B702B0156F
:101FC00009F072C209820A82A091AB03BB27AF70ED
:101FD000B02D8AE0902D0E94EB30B091AC03BF7021
:101FE000AB0FA0931402B0911502A0911402BA177E
:101FF00018F0A02DB02D02C0A1E0B02D1D01B091B0
:102000001402B01519F0A02DB02D02C0A1E0B02D22
:102010002A2A3B2A2014300411F0B1E0BA83BA8195
:10202000B01509F041C20E943529B0911402902DDB
:10203000A02D802D65DB0000A0911402BB27AA0F04
:10204000BB1FAA0FBB1FA019B24FBCD9A093170288
:10205000B09318020000A0911402BB27AA0FBB1F67
:10206000AA0FBB1FAE5FB14FADD9A0931902B093B9
:102070001A02A0911702B0911802A836FBE0BF0720
:1020800018F0A02DB02D02C0A1E0B02D1D01A0912F
:102090001702B0911802109719F4A02DB02D02C0AC
:1020A000A1E0B02D2A223B222014300419F1A09186
:1020B0001902B0911A02AA31F6E0BF0718F0A02D5C
:1020C000B02D02C0A1E0B02D1D01A0911902B09168
:1020D0001A02A035F3E0BF0718F4A02DB02D02C0FE
:1020E000A1E0B02D2A223B222014300429F4B1E0D3
:1020F000B98302C0B1E0B983000000928902009266
:102100008A02A8E6BBE0A0938B02B0938C02AFE4F6
:10211000B3E0A0938D02B0938E02AAE1B6E0A09343
:102120008F02B0939002B981B13041F400922E0237
:1021300000922F02B0E2B0931602B6C1B2E1B093A2
:102140001602B2C142D8BAE0B093F803BDE0B09332
:10215000F903BAE2B093FC03E02CA0911402BB2770
:1021600095E0AA0FBB1F9A95E1F75396AE0DB01DEF
:10217000B0D8FE01BA96EE0DF01DB083FFEFEF1A56
:10218000F8E0EF1650F3B5E0EB2EEE2DFF27F095BB
:10219000E195FF4FDE01D696EA0FFB1FB081EE2DD1
:1021A000FF27E850FC4FB083FFEFEF1AFDE0EF167A
:1021B00060F3BCE2B0930504A0911502BB27BA936B
:1021C000AA93DE015C9688E392E00E945931229640
:1021D000BB8DB0930604BA8DB0930704BCE2B093F4
:1021E0000804A0911402BB27BA93AA93DE015C965F
:1021F00088E392E00E9459312296BB8DB093090486
:10220000BA8DB0930A04BCE2B0930B04B9E5B09365
:102210000C04BCE2B0930D04B6E12AD9B0931002CD
:102220003FD9B0912902B13011F41EDC3DC1B0910B
:10223000C900B062B093C90037C10C820E94E508A2
:10224000BAE0B093F803BDE0B093F903BAE2B093FB
:10225000FC03A091AB03BB27AF70B02D8AE0902D9B
:102260000E94EB30B091AC03BF70AB0FAB83B09169
:102270001502AB81BA1718F0A02DB02D02C0A1E055
:10228000B02D1D01BB81B01519F0A02DB02D02C0DD
:10229000A1E0B02D2A2A3B2A2014300411F0B1E02D
:1022A000BC83BC81B015A9F4102DAB81BB2795E090
:1022B000AA0FBB1F9A95E1F75396A10FB01D09D83D
:1022C000FE01B296E10FF01DB0831F5F183068F376
:1022D00006C0B0E2FE01B296E10FF01DB083B5E09A
:1022E0001B2FE12FFF27F095E195FF4FDE019E9612
:1022F000EA0FFB1FB081E12FFF27E850FC4FB083AE
:102300001F5F1D3070F3BCE2B0930504B091AC03C5
:10231000B0930604B091AB03B0930704BCE2B09352
:102320000804B2E5B0930904BCE2B0930A04B3E137
:102330009FD8B0931002B4D8B0912902B13011F4F3
:1023400093DBB2C0B091C900B062B093C900ACC019
:1023500008860986202D302D0E94E508BAE0B0934A
:10236000F803BDE0B093F903BAE2B093FC030E9416
:102370004C24AB2FBB27AF73B02D1D010E949408D6
:10238000A07C2A2A3B2AD1010E9413080E949408AB
:10239000A887B987B091B202B01531F4B091B402F8
:1023A000B13019F4216001C02460B091B302B015BE
:1023B00031F4B091B502B13019F4226001C0286047
:1023C000B091B702B13009F42061B091C102B130CF
:1023D00011F4206413C0B091BE02B13011F4206832
:1023E0000DC0B091BF02B13011F4316007C0B0919F
:1023F000C002B13011F4326001C00000B091B902E6
:10240000B13009F43460B091B002B01569F4B09104
:10241000B102B01549F4B091B402B01529F4B091ED
:10242000B502B01509F43860B091C302B13009F4B7
:1024300030613A932A93DE015F9683E392E00E9433
:10244000593122960D82FE017D96BD81EB0FF01D64
:10245000B081ED81FF27F095E195FF4FE050FC4FF3
:10246000B083BD81BF5FBD83BD81B43060F3BCE28A
:10247000B0930104BFE3B0930204BCE2B093030441
:10248000BCE00E94380AB09310020AD8B091290229
:10249000B13011F4E9DA08C0B091C900B062B0936C
:1024A000C90002C0000000000E94F50800922B0243
:1024B0000092290201C055DA629B17C0B091280230
:1024C000B01599F4A0911C02B0911D02A03FF3E059
:1024D000BF0758F4B1E0B0932802AFEFB3E0A09388
:1024E0001C02B0931D02699A7198629915C0B0914F
:1024F0002802B01589F4A0911C02B0911D02AF30E2
:10250000B00551F40E9472240E9488240E9465093B
:102510000E9405090E94D6304E9943C0B0912A020C
:10252000B015F9F5B091B602B01599F4B091B902B1
:10253000B01579F4B091B702B01559F40E944C244B
:10254000B370B01531F4B4E6B0931602B1E0B093B5
:102550002A02B091B602B01521F5B091B902B015BA
:1025600001F5B091B702B015E1F40E944C24B370AC
:10257000B015B9F0B1E0B09316020092BE0200921D
:10258000BF020092C0020092C102B1E0B093B60255
:10259000B1E0B093BC02B1E0B093BD02B1E0B09342
:1025A0002A02B0913102B130D1F40E944C24AB2FF9
:1025B000BB27AF73B02D1D010E949408A07C2A2A6E
:1025C0003B2AD1010E94130800000E944C24BC70D9
:1025D000B01519F0B0E8B093160200923102B09134
:1025E0002C02B13031F40000B8E00E94213000929A
:1025F0002C02B0913002B130E9F500000E946C2449
:10260000B130A1F50000B091B702B01569F5000036
:102610000E820000AE81BB27AA0FBB1FAA0FBB1FF3
:10262000A019B24F8FEF9FEF0E94C709BE81BF5F15
:10263000BE83BE81BB3068F300000092BE020092F0
:10264000BF020092C0020092C102B1E0B093B70293
:10265000B1E0B09316020000B1E0B093BC02B1E06B
:10266000B093BD020092C302000002C00092B70204
:1026700000923002B0911602FB2FF03011F40C944E
:102680001222F13009F4BFC0F23009F4E6C0F33091
:1026900009F456C1F43009F489C1F03109F4ECC1F0
:1026A000F13109F404C2F23109F4FFC2F33109F443
:1026B00026C3F03209F420C4F13209F480C4F232A6
:1026C00009F41DC7F33209F443C7F43209F492C781
:1026D000F53211F40C94B71BF63211F40C94051C6E
:1026E000F73209F4BDC1F83211F40C94621CF932CE
:1026F00011F40C94951CFA3211F40C94D21CFB3298
:1027000011F40C941E1DFC3211F40C949B1DFD322F
:1027100011F40C94CE1DFE3211F40C940C1EFF32F9
:1027200011F40C94EB1EF03311F40C94181FF133D8
:1027300011F40C948B1FF23311F40C94BF1FF3337C
:1027400011F40C944F20F43311F40C948220F533DF
:1027500011F40C94C920F63311F40C943E1EF73397
:1027600011F40C94851EF93309F457C2FA3309F4B5
:1027700084C2F03411F40C940421F13411F40C945B
:102780004621F23411F40C948321F33411F40C94A7
:10279000BC21F03509F47FC4F13509F497C4F23552
:1027A00009F4D8C4F33509F4F0C4F43509F42FC59D
:1027B000F53509F447C5F63509F486C5F73509F44A
:1027C0009DC5F83509F4DBC5F93509F4F3C5FA35CB
:1027D00009F431C6FB3509F448C6FC3509F486C650
:1027E000FD3509F4CEC1F43609F4FDC2F53609F41D
:1027F00017C3FF3711F40C944A1CF03811F40C94F1
:1028000002220C9415220000A02DB02D0E949F24BE
:10281000A02DB02D902D0E94A924B1E0B093B90253
:102820000E944C24B1FD01C014C0A0E9B8EE902D67
:102830000E9490230E944C24AB2FBB27AF73B02D76
:102840001D010E949408A07C2A2A3B2AD1010E94E3
:102850001308B2E0B093160231CB00000E944C2462
:10286000B1FD08C00E94BD241D010E94B8242A1693
:102870003B0621F40E944C24B7FF1DC00E94722425
:102880000E944C24AB2FBB27AF73B02D1D010E94BB
:102890009408A07C2A2A3B2AD1010E941308A02D6B
:1028A000B02D0E949F24A02DB02D902D0E94A92410
:1028B000B3E0B09316020E944C24B1FD08C00E9400
:1028C000BD241D010E94B8242A163B0621F00E9457
:1028D0004C24B7FF1EC00E9472240E944C24AB2FD0
:1028E000BB27AF73B02D1D010E949408A07C2A2A3B
:1028F0003B2AD1010E941308A02DB02D0E949F24D5
:10290000A02DB02D902D0E94A924B3E0B093160203
:10291000D5CA0E94B824A039F8EEBF0709F0CECA84
:102920000E947224B4E00E9460243B2E0E9494080E
:10293000A07CA3290E941308B0E8B0931602BECA77
:102940000000A02DB02D0E94A424A02DB02D0E9427
:10295000B3240E944C24B0FD01C014C0A0E9B8EE1D
:10296000902D0E94F2230E944C24AB2FBB27AF7303
:10297000B02D1D010E949408A07C2A2A3B2AD10177
:102980000E9413080E944C24AB2FBB27AF73B02DBD
:10299000A0621D010E949408A07C2A2A3B2AD10132
:1029A0000E941308B4E0B093160288CA00000E9487
:1029B0004C24B0FD1CC00E9488240E944C24AB2FE4
:1029C000BB27AF73B02D1D010E949408A07C2A2A5A
:1029D0003B2AD1010E941308A02DB02D0E94A424EF
:1029E000A02DB02D0E94B3240092160223C00E9495
:1029F0004C24B7FBBB27B0F93B2E0E94C224A03960
:102A0000F8EEBF0719F0A02DB02D02C0A1E0B02D47
:102A1000A329109779F00E948824B8E00E946024CE
:102A20003B2E0E949408A07CA3290E941308B0E8C2
:102A3000B0931602B0911602B01509F03FCAB091DA
:102A4000B602B13011F40092B602B091B902B130C1
:102A500011F40092B90200922A020092C3022ECA17
:102A6000A0912602B0912702109709F027CAB091D1
:102A7000D002B093160222CA0000A0911702B091B2
:102A80001802902D0E9490230E944C24AB2FBB274C
:102A9000AF73B02D1D010E949408A07C2A2A3B2A06
:102AA000D1010E941308B1E1B093160207CA0000D9
:102AB000B091BD02B13051F40E944C24B1FF06C068
:102AC000A02DB02D0E949F240092BD020E944C2494
:102AD000B1FF03C0A02DB02D02C0A1E0B02D1D019B
:102AE0000E94B824A937B0051CF4A02DB02D02C057
:102AF000A1E0B02D2A223B222014300481F00E9454
:102B00007224B4E80E9460240E949408A07CA4600F
:102B1000A0680E941308B0E8B0931602CFC90E94C3
:102B2000BD241D010E94B8242A163B0691F00E9484
:102B30004C24AB2FBB27AF73B02D1D010E9494080E
:102B4000A07C2A2A3B2AF0E12F2AD1010E941308F7
:102B5000B5C90E947224BDE5B0931602B9E3B093E3
:102B6000D0020E944C24AB2FBB27AF73B02D1D01A8
:102B70000E949408A07C2A2A3B2AD1010E941308B3
:102B80009DC900000E94C224AA87BB870000A091B3
:102B90001402BB2795E0AA0FBB1F9A95E1F75D963B
:102BA0000E946909ABE0BA9FD0010024AF51BD4F2C
:102BB000AC87BD8700000E943529AA85BB858C851E
:102BC0009D85A817B90740F4B091140299E0A02D93
:102BD000802D0E94800B07C0B0911402902DA02D73
:102BE000802D0E94800B00000092C2020E941526D8
:102BF000B1E0B0932D02000001C00000B0912D02A1
:102C0000B130D9F3A8EBBBE0A0932602B093270222
:102C1000B091D002B093160251C9A0912602B09192
:102C200027021097F1F00000B0912C02B13029F486
:102C3000B8E00E94213000922C027B9B11C0B1E0D1
:102C4000B093C202B0916E00BD7FB0936E0000924F
:102C5000260200922702B0916E00B260B0936E001F
:102C60002DC9B091C202B13021F4BAE3B09316027B
:102C700025C9B6E3B093160221C90000A0EBBFE05E
:102C8000909114020E949409B1E0B093BE020092A8
:102C9000BF020092C0020092C102B02D0E944B22DE
:102CA0000E94E3250092160209C90092BE0200921A
:102CB000BF020092C002B1E0B093C10200921B02B9
:102CC00000922E0200922F020000A0911902B091F2
:102CD0001A02902D0E94F2230E944C24AB2FBB2796
:102CE000AF73B02D1D010E949408A07C2A2A3B2AB4
:102CF000D1010E941308B3E1B0931602DFC80000AF
:102D00000E944C24B170AB2FBB271D01B091BC02B7
:102D1000B13019F0A02DB02D02C0A1E0B02D2A22B3
:102D20003B222014300431F0A02DB02D0E94A424A9
:102D30000092BC020E944C24B0FF03C0A02DB02D15
:102D400002C0A1E0B02D1D010E94C224A937B00528
:102D50001CF4A02DB02D02C0A1E0B02D2A223B22F0
:102D60002014300481F00E948824B8E80E94602476
:102D70000E949408A07CA860A0680E941308B0E894
:102D8000B09316029BC80E94C7241D010E94C22452
:102D90002A163B0699F00E944C24AB2FBB27AF7339
:102DA000B02D1D010E949408A07C2A2A3B2AF0E243
:102DB0002F2AD1010E941308000080C80E94882495
:102DC000B0E1B09316020E944C24AB2FBB27AF7327
:102DD000B02D1D010E949408A07C2A2A3B2AD10113
:102DE0000E9413086BC8B1E0B093C3020000AEEDBF
:102DF000B3E0902D0E94F2230E944C24AB2FBB27FE
:102E0000AF73B02D1D010E949408A07C2A2A3B2A92
:102E1000D1010E9413080000B5E6B09316024EC817
:102E20000000B091BC02B13051F40E944C24B0FFBC
:102E300006C0A02DB02D0E94A4240092BC020E94C6
:102E40004C24B0FF03C0A02DB02D02C0A1E0B02DD6
:102E50001D010E94C224A937B0051CF4A02DB02D7D
:102E600002C0A1E0B02D2A223B222014300481F0C0
:102E70000E948824B8E80E9460240E949408A07CE4
:102E8000A860A0680E941308B0E8B093160216C8A4
:102E90000E94C7241D010E94C2242A163B06A1F0ED
:102EA0000E944C24AB2FBB27AF73B02D1D010E9495
:102EB0009408A07C2A2A3B2AF0E22F2AD1010E9402
:102EC000130800000C945E0F0E94882400921602E2
:102ED00000922A020E944C24AB2FBB27AF73B02D67
:102EE0001D010E949408A07C2A2A3B2AD1010E943D
:102EF000130800000C945E0F0092BE020092BF0205
:102F00000092C002B1E0B093C10200921B02009295
:102F10002E0200922F02B1E0B093C1020000A091F6
:102F20001902B0911A02AA31F6E0BF0718F0A02DDD
:102F3000B02D02C0A1E0B02D1D01A0911902B091E9
:102F40001A02A035F3E0BF0718F4A02DB02D02C07F
:102F5000A1E0B02D2A223B2220143004B9F0A09128
:102F60001902B0911A02902D0E94F2230E944C2463
:102F7000AB2FBB27AF73B02D1D010E949408A07C1E
:102F80002A2A3B2AD1010E94130805C0A4EAB4E012
:102F9000902D0E94F2230E944C24AB2FBB27AF73CD
:102FA000B02D1D010E949408A07C2A2A3B2AD10141
:102FB0000E941308B1E2B09316020C945E0F000059
:102FC000B091BC02B13051F40E944C24B0FF06C055
:102FD000A02DB02D0E94A4240092BC020E944C247B
:102FE000B0FF03C0A02DB02D02C0A1E0B02D1D0187
:102FF0000E94C224A937B0051CF4A02DB02D02C038
:10300000A1E0B02D2A223B222014300489F00E9436
:103010008824B8E80E9460240E949408A07CA860DC
:10302000A0680E941308B0E8B09316020C945E0FDB
:103030000E94C7241D010E94C2242A163B06A1F04B
:103040000E944C24AB2FBB27AF73B02D1D010E94F3
:103050009408A07C2A2A3B2AF0E22F2AD1010E9460
:10306000130800000C945E0F0E948824B2E2B09313
:1030700016020E944C24AB2FBB27AF73B02D1D014D
:103080000E949408A07C2A2A3B2AD1010E9413089E
:1030900000000C945E0F0000A0E8B8E0902D0E94A4
:1030A00090230E944C24AB2FBB27AF73B02D1D0182
:1030B0000E949408A07C2A2A3B2AD1010E9413086E
:1030C0000000B1E5B09316020C945E0F0000009270
:1030D0002C02B091BD02B13051F40E944C24B1FFDA
:1030E00006C0A02DB02D0E949F240092BD020E9418
:1030F000BD241D010E94B8242A163B06A1F00E949F
:103100004C24AB2FBB27AF73B02D1D010E94940838
:10311000A07C2A2A3B2AF0E12F2AD1010E94130821
:1031200000000C945E0F0E947224B2E5B093160268
:103130000E944C24AB2FBB27AF73B02D1D010E9402
:103140009408A07C2A2A3B2AD1010E94130800007F
:103150000C945E0F0000A0E6B8E091E00E9490237E
:103160000E944C24AB2FBB27AF73B02D1D010E94D2
:103170009408A07C2A2A3B2AD1010E941308B3E5B7
:10318000B093160200000C945E0F0000B091BD02D7
:10319000B13051F40E944C24B1FF06C0A02DB02DD7
:1031A0000E949F240092BD020E94BD241D010E9426
:1031B000B8242A163B06A1F00E944C24AB2FBB2753
:1031C000AF73B02D1D010E949408A07C2A2A3B2ACF
:1031D000F0E12F2AD1010E94130800000C945E0F29
:1031E0000E947224B4E5B09316020E944C24AB2FC7
:1031F000BB27AF73B02D1D010E949408A07C2A2A22
:103200003B2AD1010E94130800000C945E0F0000BD
:10321000A0E7B8E0902D0E9490230E944C24AB2F91
:10322000BB27AF73B02D1D010E949408A07C2A2AF1
:103230003B2AD1010E9413080000B5E5B0931602A5
:103240000C945E0F0000B091BD02B13051F40E94A9
:103250004C24B1FF06C0A02DB02D0E949F240092E7
:10326000BD020E94BD241D010E94B8242A163B06FF
:10327000A1F00E944C24AB2FBB27AF73B02D1D01D2
:103280000E949408A07C2A2A3B2AF0E12F2AD1012F
:103290000E94130800000C945E0F0E947224B6E591
:1032A000B09316020E944C24AB2FBB27AF73B02DF6
:1032B0001D010E949408A07C2A2A3B2AD1010E9469
:1032C000130800000C945E0F0000A1EAB4E091E046
:1032D0000E94F2230E944C24AB2FBB27AF73B02D6A
:1032E0001D010E949408A07C2A2A3B2AD1010E9439
:1032F0001308B7E5B09316020C945E0F0000B0916E
:10330000BC02B13051F40E944C24B0FF06C0A02D85
:10331000B02D0E94A4240092BC020E94C7241D016B
:103320000E94C2242A163B0699F00E944C24AB2F1F
:10333000BB27AF73B02D1D010E949408A07C2A2AE0
:103340003B2AF0E22F2AD1010E9413080C945E0F51
:103350000E948824B8E5B09316020E944C24AB2F3B
:10336000BB27AF73B02D1D010E949408A07C2A2AB0
:103370003B2AD1010E94130800000C945E0F00004C
:10338000AFE6B4E091E00E94F2230E944C24AB2F00
:10339000BB27AF73B02D1D010E949408A07C2A2A80
:1033A0003B2AD1010E9413080000B9E5B093160230
:1033B0000C945E0F0000B091BC02B13051F40E9439
:1033C0004C24B0FF06C0A02DB02D0E94A424009272
:1033D000BC020E94C7241D010E94C2242A163B067B
:1033E00099F00E944C24AB2FBB27AF73B02D1D0169
:1033F0000E949408A07C2A2A3B2AF0E22F2AD101BD
:103400000E9413080C945E0F0E948824BAE5B093C2
:1034100016020E944C24AB2FBB27AF73B02D1D01A9
:103420000E949408A07C2A2A3B2AD1010E941308FA
:1034300000000C945E0F0000A8E8B4E091E00E9448
:10344000F2230E944C24AB2FBB27AF73B02D1D017C
:103450000E949408A07C2A2A3B2AD1010E941308CA
:10346000BBE5B09316020C945E0F0000B091BC0255
:10347000B13051F40E944C24B0FF06C0A02DB02DF5
:103480000E94A4240092BC020E94C7241D010E9435
:10349000C2242A163B0699F00E944C24AB2FBB276E
:1034A000AF73B02D1D010E949408A07C2A2A3B2AEC
:1034B000F0E22F2AD1010E9413080C945E0F0E94A3
:1034C0008824B5E3B09316020E944C24AB2FBB278F
:1034D000AF73B02D1D010E949408A07C2A2A3B2ABC
:1034E000D1010E94130800000C945E0FF894A89577
:1034F000B9E3B09360000000FECF0C945E0F0000B3
:10350000B091B802B01541F4A0918B02B0918C0239
:10351000902D0E94902307C0A0918902B0918A0249
:10352000902D0E9490230E944C24AB2FBB27AF7399
:10353000B02D1D010E949408A07C2A2A3B2AD101AB
:103540000E9413080000B3E2B09316020C945E0FC1
:103550000000B0912C02B13061F4B8E00E9421303B
:10356000B01511F4000003C0B8E2B0931602009247
:103570002C02B091BD02B13051F40E944C24B1FF35
:1035800006C0A02DB02D0E949F240092BD020E9473
:10359000BD241D010E94B8242A163B06A1F00E94FA
:1035A0004C24AB2FBB27AF73B02D1D010E94940894
:1035B000A07C2A2A3B2AF0E12F2AD1010E9413087D
:1035C00000000C945E0F0E947224B4E2B0931602C5
:1035D0000E944C24AB2FBB27AF73B02D1D010E945E
:1035E0009408A07C2A2A3B2AD1010E9413080000DB
:1035F0000C945E0F0000B091B802B01521F4B1E058
:10360000B093B80202C00092B8020E94C224809116
:103610008F0290919002A817B9071CF0B1E0B09307
:103620002E02A0918D02B0918E021D010E94C22433
:103630002A163B061CF0B1E0B0932F020000B091B7
:10364000B802B01521F4B0912E02B01541F0B0913E
:103650002F02B13031F5B0912E02B01511F50E9454
:10366000C72490911B0286E1989FC0010024A80FF7
:10367000B91FAE87BF870000AE85BF85902D0E9421
:10368000F2230E944C24AB2FBB27AF73B02D1D013A
:103690000E949408A07C2A2A3B2AD1010E94130888
:1036A00031C0B091B802B13021F4B0912F02B01501
:1036B00041F0B0912E02B13029F5B0912F02B01532
:1036C00009F50E94C72490911B0286E1989FC001D2
:1036D0000024A81BB90BAE87BF870000AE85BF854D
:1036E000902D0E94F2230E944C24AB2FBB27AF7376
:1036F000B02D1D010E949408A07C2A2A3B2AD101EA
:103700000E9413080000B5E2B0931602B0912E0299
:10371000B130C9F4B0912F02B130A9F4BFE7B09332
:1037200016020E944C24AB2FBB27AF73B02D1D0196
:103730000E949408A07C2A2A3B2AD1010E941308E7
:1037400000000C945E0FB0912E02B13021F0B091C8
:103750002F02B13029F4B1E0B0931B020C945E0F3C
:10376000B0911B02BF5FB0931B020C945E0F000070
:103770000E944C24B170AB2FBB271D01B091BC023D
:10378000B13019F0A02DB02D02C0A1E0B02D2A2239
:103790003B222014300431F0A02DB02D0E94A4242F
:1037A0000092BC020E94C7241D010E94C2242A1656
:1037B0003B06A1F00E944C24AB2FBB27AF73B02D6A
:1037C0001D010E949408A07C2A2A3B2AF0E22F2A9D
:1037D000D1010E94130800000C945E0F0E948824FF
:1037E000B6E2B09316020E944C24AB2FBB27AF73F6
:1037F000B02D1D010E949408A07C2A2A3B2AD101E9
:103800000E94130800000C945E0F00000E94C22466
:10381000A88BB98B0000A0911402BB2795E0AA0FDA
:10382000BB1F9A95E1F75D960E946909ABE0BA9FCC
:10383000D0010024AF51BD4FAA8BBB8B0000A889DB
:10384000B9898A899B89A817B90740F4B0911402F5
:1038500099E0A02D802D0E94800B07C0B09114022A
:10386000902DA02D802D0E94800BB2E2B093160205
:103870000E944C24AB2FBB27AF73B02D1D010E94BB
:103880009408A07C2A2A3B2AD1010E941308000038
:103890000C945E0F00000092BE02B1E0B093BF0234
:1038A0000092C0020092C102A2E6B2E0A0932602FA
:1038B000B0932702B1E0B093D002B7E2B093160202
:1038C0000C945E0F00000E94B8246D010000B091BE
:1038D000B802B01529F4F0EACF1AFFEFDF0A03C0EF
:1038E000F0E6CF1AD008A0918B02B0918C02AC15F3
:1038F000BD052CF4A0918B02B0918C026D01A091BA
:103900008902B0918A02CA16DB062CF4A0918902C2
:10391000B0918A026D01D60191E00E94A9240000B5
:10392000B9E2B09316020C945E0F0000B091BD0294
:10393000B13041F4B1D7B1FF05C0A02DB02DFFD7F4
:103940000092BD020E94BD241D010E94B8242A16C7
:103950003B0699F0A1D7AB2FBB27AF73B02D1D014C
:103960000E949408A07C2A2A3B2AF0E12F2AD10148
:103970000E94130800000C945E0FB4D7BAE2B09313
:1039800016028AD7AB2FBB27AF73B02D1D010E9443
:103990009408A07C2A2A3B2AD1010E941308000027
:1039A0000C945E0F0000E4D7FA2E0B2F0092200239
:1039B00000922102F0921E0200931F02B091B80201
:1039C000B13021F4F0E4FF1A0F4F03C0F0ECFF1AFE
:1039D0000009A0918B02B0918C02AF15B00734F4AE
:1039E000A0918B02B0918C02FA2E0B2FA09189022C
:1039F000B0918A02FA160B0734F4A0918902B091B3
:103A00008A02FA2E0B2FB02FAF2D91E089D644D722
:103A1000AB2FBB27AF73B02D1D010E949408A07C73
:103A20002A2A3B2AD1010E9413080000BBE2B0936E
:103A30001602B0E4B093D1020C945E0F0000B09176
:103A40002C02B130F1F5B8E00E942130B01519F523
:103A5000A0912002B0912102109789F1B091D1027A
:103A6000B150B093D102B091D102B01541F53AD71F
:103A7000BCE2B093160210D7AB2FBB27AF73B02DAB
:103A80001D010E949408A07C2A2A3B2AD1010E9491
:103A90001308000014C0B0E4B093D102A09120023A
:103AA000B0912102109731F463D7A0932002B09314
:103AB000210205C05DD7A0931E02B0931F020092A1
:103AC0002C02B091BD02B13041F4E6D6B1FF05C081
:103AD000A02DB02D34D70092BD024FD71D0148D77D
:103AE0002A163B0699F0D8D6AB2FBB27AF73B02D63
:103AF0001D010E949408A07C2A2A3B2AF0E12F2A6B
:103B0000D1010E94130800000C945E0FEBD6BCE2BA
:103B1000B0931602C1D6AB2FBB27AF73B02D1D01DA
:103B20000E949408A07C2A2A3B2AD1010E941308F3
:103B300000000C945E0F0000A0912002B0912102C1
:103B4000109741F4A0911E02B0911F02A093200291
:103B5000B0932102A0912002B091210280911E0217
:103B600090911F02A80FB91F82E0902D0E94D830BB
:103B7000902DD6D591D6AB2FBB27AF73B02D1D019D
:103B80000E949408A07C2A2A3B2AD1010E94130893
:103B90000000BDE2B09316020C945E0F0000B091DD
:103BA000BD02B13041F478D6B1FF05C0A02DB02DD3
:103BB000C6D60092BD02E1D61D01DAD62A163B0612
:103BC00099F06AD6AB2FBB27AF73B02D1D010E94B1
:103BD0009408A07C2A2A3B2AF0E12F2AD1010E94D6
:103BE000130800000C945E0F7DD6BDE5B09316025D
:103BF000BEE2B093D00250D6AB2FBB27AF73B02D2F
:103C00001D010E949408A07C2A2A3B2AD1010E940F
:103C1000130800000C945E0FA0912602B0912702B9
:103C20001097F1F00000B0912C02B13029F4B8E007
:103C30000E94213000922C027B9B11C0B1E0B09316
:103C4000C202B0916E00BD7FB0936E00009226025A
:103C500000922702B0916E00B260B0936E000BC06C
:103C6000B091C202B13021F4BFE2B093160203C09A
:103C7000B6E3B093160200000C945E0F000078D6F5
:103C80005D01B091B802B01529F4F0EDAF1AFFEF65
:103C9000BF0A03C0F0E3AF1AB008B091B802B01584
:103CA00069F4A0918B02B0918C02AA15BB0594F423
:103CB000A0918B02B0918C025D010CC0A091890291
:103CC000B0918A02AA16BB062CF4A0918902B09189
:103CD0008A025D010000D50191E022D5DDD5AB2F30
:103CE000BB27AF73B02D1D010E949408A07C2A2A27
:103CF0003B2AD1010E9413080000B0E4B093D10226
:103D0000B7E3B09316020C945E0F0000B091BD02B1
:103D1000B13041F4C1D5B1FF05C0A02DB02D0FD6F3
:103D20000092BD022AD61D0123D62A163B0629F190
:103D3000B3D5AB2FBB27AF73B02D1D010E949408E4
:103D4000A07C2A2A3B2AF0E12F2AD1010E941308E5
:103D5000B0912C02B13021F5B8E00E942130B015AD
:103D600031F4B091D102B150B093D10203C0B0E4AC
:103D7000B093D10200922C0213C0B4D5B2E2B0933A
:103D800016028AD5AB2FBB27AF73B02D1D010E9441
:103D90009408A07C2A2A3B2AD1010E941308000023
:103DA000B091D102B01511F00C945E0F9BD5B2E228
:103DB000B093160271D5AB2FBB27AF73B02D1D0189
:103DC0000E949408A07C2A2A3B2AD1010E94130851
:103DD00000000C945E0F0000D5D52D01F0E44F1AC1
:103DE000FFEF5F0AA0918F02B0919002A415B50574
:103DF0002CF4A0918F02B09190022D010000D2010D
:103E000091E0F0D449D5AB2FBB27AF73B02D1D0186
:103E10000E949408A07C2A2A3B2AD1010E94130800
:103E2000B0E4B093D102B0E3B09316020C945E0FED
:103E3000000032D5B170AB2FBB271D01B091BC0281
:103E4000B13019F0A02DB02D02C0A1E0B02D2A2272
:103E50003B222014300429F0A02DB02D75D50092FE
:103E6000BC0295D51D018ED52A163B0691F014D5BE
:103E7000AB2FBB27AF73B02D1D010E949408A07C0F
:103E80002A2A3B2AF0E22F2AD1010E9413080000BF
:103E900013C03ED5B1E3B0931602FED4AB2FBB27BF
:103EA000AF73B02D1D010E949408A07C2A2A3B2AE2
:103EB000D1010E9413080000B0912C02B13011F022
:103EC0000C945E0FB8E00E942130B015E9F4B09177
:103ED000D102B150B093D102B091D102B015B9F472
:103EE00017D5B1E3B0931602D7D4AB2FBB27AF736E
:103EF000B02D1D010E949408A07C2A2A3B2AD101E2
:103F00000E941308000003C0B0E4B093D1020092F5
:103F10002C020C945E0F000035D53D01F0EC6F1AB9
:103F20007008A0918D02B0918E026A167B062CF467
:103F3000A0918D02B0918E023D016092220270929A
:103F4000230200922402009225020000D30191E096
:103F500049D4A2D4AB2FBB27AF73B02D1D010E9453
:103F60009408A07C2A2A3B2AD1010E941308B0E4BD
:103F7000B093D102B2E3B09316020C945E0F00002E
:103F8000B0912C02B13009F044C00000B8E00E94AA
:103F90002130B01531F50000A0912402B091250226
:103FA0001097E9F00000B091D102B150B093D10266
:103FB000B091D102B01599F4ABD4B3E3B09316022B
:103FC0006BD4AB2FBB27AF73B02D1D010E9494089B
:103FD000A07C2A2A3B2AD1010E941308000000007D
:103FE00016C0B0E4B093D1020000A0912402B091B9
:103FF0002502109731F4C6D4A0932402B093250271
:1040000005C0C0D4A0932202B09323020000009206
:104010002C0242D4B170AB2FBB271D01B091BC0262
:10402000B13019F0A02DB02D02C0A1E0B02D2A2290
:104030003B222014300429F0A02DB02D85D400920D
:10404000BC02A5D41D019ED42A163B0699F024D4A7
:10405000AB2FBB27AF73B02D1D010E949408A07C2D
:104060002A2A3B2AF0E22F2AD1010E9413080000DD
:104070000C945E0F4DD4B3E3B09316020DD4AB2F66
:10408000BB27AF73B02D1D010E949408A07C2A2A83
:104090003B2AD1010E94130800000C945E0F00001F
:1040A000A0912402B0912502109741F4A091220220
:1040B000B0912302A0932402B09325020000A091A6
:1040C0002402B09125028091220290912302A80F30
:1040D000B91F82E0902D0E94D830902D83D3DCD37D
:1040E000AB2FBB27AF73B02D1D010E949408A07C9D
:1040F0002A2A3B2AD1010E941308B4E3B093160286
:104100000C945E0F0000C8D3B170AB2FBB271D010C
:10411000B091BC02B13019F0A02DB02D02C0A1E0C9
:10412000B02D2A223B222014300429F0A02DB02DDE
:104130000BD40092BC022BD41D0124D42A163B06BA
:1041400099F0AAD3AB2FBB27AF73B02D1D010E94EE
:104150009408A07C2A2A3B2AF0E22F2AD1010E944F
:10416000130800000C945E0FD3D3B5E3B09316028E
:1041700093D3AB2FBB27AF73B02D1D010E949408C2
:10418000A07C2A2A3B2AD1010E94130800000C942B
:104190005E0F0000EDD3AC8BBD8BA0911402BB274A
:1041A000AA0FBB1FAA0FBB1FA019B24F8C899D89F4
:1041B0000E94C7090000E6D3AC8BBD8BA09114020E
:1041C000BB27AA0FBB1FAA0FBB1FAE5FB14F8C89C5
:1041D0009D890E94C7090000A0EBBFE090911402E6
:1041E0000E9494090000B02D56D1EDD4B1E0B093F7
:1041F000BE020092BF020092C0020092C102009271
:10420000160200000C945E0F00000092BE020092A5
:10421000BF02B1E0B093C0020092C102B091B402FB
:10422000B13079F5A5D34D01B7D3B01529F4F0EA33
:104230008F1AFFEF9F0A03C0F0E68F1A9008A09133
:104240008B02B0918C02A815B9052CF4A0918B02B9
:10425000B0918C024D01A0918902B0918A028A1618
:104260009B062CF4A0918902B0918A024D010000B6
:10427000D40191E06ED30000B1E4B09316020C9427
:104280005E0FB2E4B09316020C945E0F0000B09182
:10429000BD02B13051F400D3B1FF07C00000A02D22
:1042A000B02D4DD300000092BD0267D31D0160D335
:1042B0002A163B0699F0F0D2AB2FBB27AF73B02D77
:1042C0001D010E949408A07C2A2A3B2AF0E12F2A93
:1042D000D1010E94130800000C945E0F03D3B2E4D6
:1042E000B0931602D9D2AB2FBB27AF73B02D1D01EF
:1042F0000E949408A07C2A2A3B2AD1010E9413081C
:1043000000000C945E0F0000B091B502B13071F561
:1043100000003DD3A88FB98F000034D3AE8BBF8B84
:104320000000AE89BF89888D998DA817B9077CF4E4
:10433000A88DB98D8E899F89A81BB90BA136B005B0
:10434000A4F0AE89BF89A05ABF4F0DD30EC0AE896D
:10435000BF89888D998DA81BB90BA136B0052CF0AB
:10436000AE89BF89A056B009FED20000B3E4B09375
:10437000160200000C945E0F00008ED2B170AB2FBD
:10438000BB271D01B091BC02B13019F0A02DB02D9A
:1043900002C0A1E0B02D2A223B222014300429F0D3
:1043A000A02DB02DD1D20092BC02F1D21D01EAD2D3
:1043B0002A163B0699F070D2AB2FBB27AF73B02DF6
:1043C0001D010E949408A07C2A2A3B2AF0E22F2A91
:1043D000D1010E94130800000C945E0F99D2009244
:1043E00016025AD2AB2FBB27AF73B02D1D010E940E
:1043F0009408A07C2A2A3B2AD1010E9413080000BD
:104400000C945E0FB9E3BF830000B1E0B0933202B9
:10441000000068D200007CD200000092160200006A
:104420000C945E0F00000C945E0F009216020C9428
:104430005E0FE396089501C00000B0E18BD0B1306B
:10444000D9F3B0914202B36C60D092C008953A9310
:104450003B2F301531F4B0914202BF7DB093420240
:1044600005C0B0914202B062B0934202E6DF3991DA
:1044700008953A933B2F301531F4B0914202B77F43
:10448000B093420205C0B0914202B860B0934202BC
:10449000D4DF399108953A933B2F301531F4B09120
:1044A0004202BB7FB093420205C0B0914202B460A9
:1044B000B0934202C2DF39910895B0914202B2FF37
:1044C00002C0B1E00895B02D0895B02DBCEFAAB19F
:1044D000AB23AAB90895B01511F4599801C0599A9F
:1044E000519A589A509A509801C00000489BFDCFAD
:1044F0005898509A08955198589A509A499902C0DC
:10450000B02D01C0B1E0589808953A932A932B2F0B
:10451000302D27FBBB27B0F9DEDF220F3F5F38309D
:10452000C0F30000E8DF2991399108953A932A9366
:104530001A931B2F202D302D04C0330FDCDF3B2BB3
:104540002F5F2830D0F3B12FC6DFB32F19912991F7
:10455000399108953A933B2F589A599A509A0000EE
:10456000519A000059985898B32FCFDF3991089588
:10457000589800005998509A0000519A0000589A93
:104580000000599A0895B0302CF4CD019095819592
:104590009F4FDC010895B0916A00B07FB960B0937D
:1045A0006A006E9857985498BFEFB1B9259A009257
:1045B0008800B0918000B168B0938000B091810014
:1045C000B160B0938100BBE0B09391000092920083
:1045D000BFE3B0939900BFEFB0939800B2E0B093FF
:1045E00071000895A02DB02D00001196AF3FFFE798
:1045F000BF07D0F3089500009091440293FF4EC08E
:10460000009288009FEF92B900924502A02DB02D34
:10461000000000000000000000000000000000009A
:10462000000000000000000000000000000000008A
:10463000000000000000000000000000000000007A
:10464000000000000000000000000000000000006A
:10465000000000000000000000000000000000005A
:10466000000000000000000000000000000000004A
:10467000000000000000000000000000000000003A
:104680001196AF3FFFE7BF0718F2EC98ED989091B5
:1046900071009D7F9093710002B80895909144023B
:1046A00090FF0AC09091440291FF03C092E092B93A
:1046B0000CC091E092B909C09091440291FF03C0EF
:1046C00090E292B902C090E192B900924502A02D09
:1046D000B02D0000000000000000000000000000FD
:1046E0000000000000000000000000000000119623
:1046F000AF3FFFE7BF0768F390915102901519F49F
:104700000092880004C0909150029093880090918C
:10471000710092609093710092B19C6C92B908956F
:104720003A932A931A939D01192F0000B0914402E5
:10473000B860B09344025FDFB0914302BF7EB09394
:1047400043020000A0914B02B0914C02A217B307A4
:1047500009F444C00000A0914702B09148022A1712
:104760003B073CF0B0914402B87FBA5FB09344027B
:1047700006C0B0914402B87FBC5FB0934402A091E0
:104780004702B0914802A21BB30BFDDEA03BB0056F
:104790002CF4B0914402BB7FB0934402000011306E
:1047A00049F4B0914402BB7FB0934402B1E0B093AE
:1047B000510202C00092510220934B0230934C02EE
:1047C00000924602B0914402B77FB0934402EC9A43
:1047D00012DFB0914302B061B09343021991299165
:1047E000399108953A932A931A939D01192F000045
:1047F000B0914402B860B0934402FDDEB091430230
:10480000BF7DB0934302A0914D02B0914E02A2171A
:10481000B307F1F10000A0914902B0914A022A17B2
:104820003B073CF0B0914402B87FB95FB0934402BB
:1048300006C0B0914402B87FBB5FB0934402A09120
:104840004902B0914A02A21BB30B9DDEA438B00509
:104850002CF4B0914402BB7FB093440200001130AD
:1048600029F4B0914402BB7FB093440220934D02DF
:1048700030934E0200924602B0914402B77FB0934B
:104880004402ED9AB8DEB0914302B062B0934302A5
:104890001991299139910895B02D0000669B01C0AE
:1048A000B2604F9B01C0B1600000AB2F90914302FA
:1048B0009C7FA90FA0934302A0914302BA2F0895B1
:1048C0003A933B2FB32FA0914302AF7DBA2BB09305
:1048D0004302E2DF399108954C9B02C0B02D089548
:1048E000B1E008950000B0914402B860B093440272
:1048F00082DEB0914302BF7EB093430273DEA0918B
:104900004702B0914802A0934B02B0934C02089525
:104910000000B0914402B860B09344026CDEB091E4
:104920004302BF7DB09343025DDE0000A0914902C7
:10493000B0914A02A0934D02B0934E020895A09305
:104940004702B09348020895A0934902B0934A02E7
:104950000895913019F480E280934F02A0934B02A6
:10496000B0934C020895A0934D02B0934E02089567
:10497000A0914702B09148020895A0914B02B091D6
:104980004C020895A0914902B0914A020895A09165
:104990004D02B0914E020895B0914402B1FF02C0A1
:1049A000B02D0895B1E00895CD0101C001970097A1
:1049B000E9F708955598A02DB0ECF6DF559A0895C3
:1049C0003A932A931A9322979D01192F01C0000050
:1049D000EAE6FAE0B491BEDDB130C9F3F901EE0FB9
:1049E000FF1FEE5EFE4FA591B591A883B983B981F3
:1049F0008CDDB8818ADDB12F88DDBADD2296199170
:104A00002991399108953A932A931A9322971A2F4C
:104A10002B2F01C00000EAE6FAE0B4919BDDB13033
:104A2000C9F3F22FE12FEE0FFF1FEE5EFE4FA591AF
:104A3000B591A883B983B98168DDB88166DD98DD59
:104A400001C00000EAE6FAE0B491B16083DDB13064
:104A5000C1F3B1E06BDD3B2F8BDDB32F22961991B3
:104A60002991399108953A932A933B2F2A2F01C017
:104A70000000E5E7FAE0B4916DDDB130C9F3B32F82
:104A800044DDB22F42DD74DD2991399108953A93C6
:104A90002A932B2F01C00000E5E7FAE0B4915ADD1C
:104AA000B130C9F3B22F31DD63DD01C00000E5E7AD
:104AB000FAE0B491B1604EDDB130C1F3B1E036DD62
:104AC0003B2F56DDB32F2991399108953A932A93BC
:104AD0001A930A93FA92EA92DA92CA92BA92AA9234
:104AE0009A928A924C015D01A5E3B02D8CDFB5FD51
:104AF00003C0A6E0B02D02C0A4E0B02DCD01AA27CE
:104B000097FDA095BA2F6C017D01D701C601B501B3
:104B1000A4010E94F430EBE6FAE0459155916591CD
:104B200075910E942B310197A009B0098C019D015C
:104B3000B02F89909990A990B990C990D990E99097
:104B4000F990099119912991399108953A932A93ED
:104B50001A930A93FA92EA92DA92CA92BA92BB2E06
:104B6000A5E3B02D50DFB5FD03C0A6E0B02D02C017
:104B7000A4E0B02DCD01AA2797FDA095BA2F6C0116
:104B80007D018B2D9927AA27BB278F5F9F4FAF4FA2
:104B9000BF4FEBE6FAE045915591659175910E9402
:104BA000F430B701A6010E942B318C019D01D9017F
:104BB000C801B990C990D990E990F99009911991DB
:104BC0002991399108953A93A5E3B02D1CDF3B2F2D
:104BD00037FD05C0A5E3B02D932F9068F1DEABE360
:104BE000B02D11DF3B2F31FF05C0ABE3B02D932F6C
:104BF0009D7FE6DE399108953A93A5E3B02D03DF5A
:104C00003B2F37FF05C0A5E3B02D932F9F77D8DE4C
:104C1000ABE3B02DF8DE3B2F31FD05C0ABE3B02D8B
:104C2000932F9260CDDE399108953A93A8E6B1E0D2
:104C3000EADE3B2FA8E6B1E0932F9E7FC1DEA02DD8
:104C4000B0E6B2DEA8E6B1E0DEDE3B2FA8E6B1E0DA
:104C5000932F9160B5DEA8E6B1E0D5DE3B2FA8E644
:104C6000B1E0932F9E7FACDE399108953A932A9359
:104C70001A930A93FA92EA92EB2E202D302DBBE084
:104C8000FB2EFE2DF03031F0F13039F0F23049F0EA
:104C9000F33059F0202D302D0BC0A1E0BB279D0132
:104CA00007C0A2E0BB279D0103C0A3E0BB279D0175
:104CB000B0915C04B03320F0AAE2BAE08D0107C0E5
:104CC000B0915C04B03218F0A6E4BAE08D01A09176
:104CD0009502B0919602A93BFBE0BF0758F4D901B9
:104CE00087E0902D0E94EB30A00FB11FFD01B28133
:104CF000FB2E43C0A0919502B0919602A935FBE12D
:104D0000BF0758F4D90187E0902D0E94EB30A00F27
:104D1000B11FFD01B381FB2E30C0A0919502B0916F
:104D20009602A939FAE3BF0758F4D90187E0902D1C
:104D30000E94EB30A00FB11FFD01B481FB2E1DC0FE
:104D4000A0919502B0919602A93AF1E6BF0758F4F6
:104D5000D90187E0902D0E94EB30A00FB11FFD011B
:104D6000B581FB2E0AC0D90187E0902D0E94EB305F
:104D7000A00FB11FFD01B681FB2EBF2DE990F99068
:104D8000099119912991399108953A932A931A9387
:104D90000A93FA92EA92DA92CA92BA92AA929A92F2
:104DA0008A927A92AB2E9A2EB9E21B2FB0915C04B4
:104DB000B03269F4AAE8B7E0FA2E0B2FA2EEB9E000
:104DC000DA2EEB2EAAEDB8E0BA2ECB2E0CC0A2E361
:104DD000B8E0FA2E0B2FA6E0BAE0DA2EEB2EAEE505
:104DE000B9E0BA2ECB2EF4E0AF1600F5202D302D11
:104DF00002C02F5F3F4F233030058CF4AA2DBB2714
:104E00007A2E8B2ED9018CE0902D0E94EB30AD0DC7
:104E1000BE1DFD01A591B5917A168B0651F7233081
:104E20003005FCF1A2E0BB279D013BC0202D302DB9
:104E300002C02F5F3F4F2E3030058CF4AA2DBB27C8
:104E40007A2E8B2ED9018CE0902D0E94EB30AF0D85
:104E5000B01FFD01A591B5917A168B0651F72E3042
:104E60003005FCF0202D302D02C02F5F3F4F2B303E
:104E700030058CF4AA2DBB277A2E8B2ED9018CE01D
:104E8000902D0E94EB30AB0DBC1DFD01A591B5919D
:104E90007A168B0651F72B3030051CF0AAE0BB27A1
:104EA0009D01F4E0AF1608F0BBC0901409F45CC09B
:104EB000A0919502B0919602A93BFBE0BF0760F478
:104EC000D9018CE0902D0E94EB30AD0DBE1D1296E5
:104ED000FD01B4911B2FBAC1A0919502B091960229
:104EE000A935FBE1BF0760F4D9018CE0902D0E9449
:104EF000EB30AD0DBE1D1496FD01B4911B2FA6C164
:104F0000A0919502B0919602A939FAE3BF0760F427
:104F1000D9018CE0902D0E94EB30AD0DBE1D169690
:104F2000FD01B4911B2F92C1A0919502B091960200
:104F3000A93AF1E6BF0760F4D9018CE0902D0E94F8
:104F4000EB30AD0DBE1D1896FD01B4911B2F7EC137
:104F5000D9018CE0902D0E94EB30AD0DBE1D1A964C
:104F6000FD01B4911B2F72C1A0919502B0919602E0
:104F7000A93BFBE0BF0760F4D9018CE0902D0E94B3
:104F8000EB30AD0DBE1D1396FD01B4911B2F5EC11C
:104F9000A0919502B0919602A935FBE1BF0760F49C
:104FA000D9018CE0902D0E94EB30AD0DBE1D159601
:104FB000FD01B4911B2F4AC1A0919502B0919602B8
:104FC000A939FAE3BF0760F4D9018CE0902D0E9463
:104FD000EB30AD0DBE1D1796FD01B4911B2F36C1F0
:104FE000A0919502B0919602A93AF1E6BF0760F44C
:104FF000D9018CE0902D0E94EB30AD0DBE1D1996AD
:10500000FD01B4911B2F22C1D9018CE0902D0E948B
:10501000EB30AD0DBE1D1B96FD01B4911B2F16C1CB
:10502000F2E1AF1608F0BBC0901409F45CC0A09187
:105030009502B0919602A93BFBE0BF0760F4D9014D
:105040008CE0902D0E94EB30AF0DB01F1296FD0149
:10505000B4911B2FFBC0A0919502B0919602A93587
:10506000FBE1BF0760F4D9018CE0902D0E94EB308A
:10507000AF0DB01F1496FD01B4911B2FE7C0A09196
:105080009502B0919602A939FAE3BF0760F4D901FD
:105090008CE0902D0E94EB30AF0DB01F1696FD01F5
:1050A000B4911B2FD3C0A0919502B0919602A93A5A
:1050B000F1E6BF0760F4D9018CE0902D0E94EB303F
:1050C000AF0DB01F1896FD01B4911B2FBFC0D901C1
:1050D0008CE0902D0E94EB30AF0DB01F1A96FD01B1
:1050E000B4911B2FB3C0A0919502B0919602A93B39
:1050F000FBE0BF0760F4D9018CE0902D0E94EB30FB
:10510000AF0DB01F1396FD01B4911B2F9FC0A0914E
:105110009502B0919602A935FBE1BF0760F4D90171
:105120008CE0902D0E94EB30AF0DB01F1596FD0165
:10513000B4911B2F8BC0A0919502B0919602A93912
:10514000FAE3BF0760F4D9018CE0902D0E94EB30A8
:10515000AF0DB01F1796FD01B4911B2F77C0A09122
:105160009502B0919602A93AF1E6BF0760F4D90121
:105170008CE0902D0E94EB30AF0DB01F1996FD0111
:10518000B4911B2F63C0D9018CE0902D0E94EB30AD
:10519000AF0DB01F1B96FD01B4911B2F57C0A091FE
:1051A0009502B0919602A93BFBE0BF0760F4D901DC
:1051B0008CE0902D0E94EB30AB0DBC1D1296FD01D2
:1051C000B4911B2F43C0A0919502B0919602A935CE
:1051D000FBE1BF0758F4D9018CE0902DFCD7AB0D53
:1051E000BC1D1496FD01B4911B2F30C0A0919502F7
:1051F000B0919602A939FAE3BF0758F4D9018CE0BF
:10520000902DE9D7AB0DBC1D1696FD01B4911B2F57
:105210001DC0A0919502B0919602A93AF1E6BF0790
:1052200058F4D9018CE0902DD6D7AB0DBC1D189643
:10523000FD01B4911B2F0AC0D9018CE0902DCBD772
:10524000AB0DBC1D1A96FD01B4911B2FB12F7990A7
:1052500089909990A990B990C990D990E990F990C6
:10526000099119912991399108953A932A931A93A2
:105270002297A0DBA02DB02DC6DBB0935C04A8E77D
:10528000B02D9CE19DDBA02DB0EC8EDBA5E3B02D15
:10529000BADBB0629B2FA5E3B02D92DBAFE8B1E0A3
:1052A0009CE68EDBADE0B02D90E48ADBEFE6FAE021
:1052B00085919591A591B59109DC9B2FA4E3B02D23
:1052C0007FDBA02DB0EC70DBACE0B02D99E078DB9B
:1052D000A5E3B02D92E274DBA02DB0EC65DBA7E373
:1052E000B02D91DB1B2FADE0B02D90EC69DBB02D24
:1052F000A0915202B8DBB1E0A0915302B4DBADE063
:10530000B02D90E45DDB202D302DF901EE0FFF1F55
:10531000E25BFB4FB491B130D9F401C00000B0EDB5
:1053200019D9B130D9F3F901EE0FFF1FEE5EFE4F30
:10533000A591B591A883B983B981E7D8B881E5D89B
:10534000F901EE0FFF1FE15BFB4FB491DED810D9DE
:1053500000002F5F3F4F2E39F1E03F07B0F2000011
:10536000A4E3B02D50DBF2DBE8E5F4E08083918329
:10537000A283B383A7E6B1E090EB22DBA8E6B1E01D
:1053800090E81EDBA9E6B1E0902D1ADBAAE6B1E0B9
:1053900090E216DBABE6B1E0902D12DBACE6B1E0BB
:1053A00093E00EDBADE6B1E0902D0ADBAEE6B1E0B6
:1053B00099E606DB229619912991399108953A933D
:1053C0002A931A930A93FA92EA92DA92CA92000006
:1053D000A0919F02B091A0028091910290919202BF
:1053E000A817B90760F4A0919102B0919202809140
:1053F0009D0290919E02A81BB90B7D010BC0A0914C
:105400009102B091920280919B0290919C02A81B04
:10541000B90B7D01F4E0FF1620F4B0E5B09355021E
:1054200015C0F5E1EF16F5E0FF0620F4B0E7B09304
:1054300055020CC0FFEFEF16F7E0FF0620F4B0E8CE
:10544000B093550203C0B0EAB0935502E092540203
:10545000D701AB2FBB27AF70B0915502B07FAB2BFC
:10546000A0935502B0919A02FB2FF53139F1F83132
:1054700009F04EC0A0919502B09196028D01202DA9
:10548000302DD901C80143E2502D602D702DACD6CE
:1054900044E6502D602D702DDED6080F191F2A1FEF
:1054A0003B1FD901C801805F984DAF4FBF4FB695E4
:1054B000A795979587958C019D0130C0A091950285
:1054C000B09196028D01202D302DD901C80143E203
:1054D000502D602D702D88D644E6502D602D702DF6
:1054E000BAD6080F191F2A1F3B1FD901C8014EE168
:1054F000502D602D702D78D680529C46AB4FBF4FFB
:1055000048E2502D602D702DA6D68C019D0106C05D
:1055100080EA9CE8AA27BB278C019D01013AFCE8A0
:105520001F072005300538F0B0915602B07EBF61EC
:10553000B09356021AC00838F3E11F072005300562
:1055400030F4B0915602B07EB09356020EC0D9012D
:10555000C80148EE53E0602D702D7DD68550B09186
:105560005602B07E8B2B80935602ADE0B02D90ECAE
:1055700027DAB2E0A091540276DAB3E0A0915502A6
:1055800072DAB4E0A09156026EDAB0915702B260BE
:10559000B0935702A02DB0E207DAB0915702B46081
:1055A000B0935702B5E0A09157025DDAC02CD02C21
:1055B000B5E06DDAB2FD01C00BC0A02DB0E2F4D9A8
:1055C000FFEFCF1AFFEFDF0AFAE0CF16D00480F327
:1055D000ADE0B02D90E4F4D9C990D990E990F9905C
:1055E000099119912991399108953A932A931A931F
:1055F0000A93FA922697A8E7B02D9FE1E1D9B091DE
:105600005C04B03220F0A0E8B02D9EE9D9D9A9E71A
:10561000B02D90E2D5D9ADE9B02D92EDD1D9A091C0
:105620009502B0919602A13DF7E0BF0728F4AFE7DD
:10563000B02D93E6C5D904C0AFE7B02D90E7C0D92F
:10564000A5E8B02D98E3BCD9B0915C04B03220F04D
:10565000A4EAB02D9AE5B4D9A6EAB02D902DB0D920
:10566000A0919502B0919602AA83BB830C820D8211
:105670008A819B81AC81BD81B92FA82F992788276A
:105680008A839B83AC83BD83E8E5F4E080819181CC
:10569000A281B38148EE53E0602D702DDCD5AC01C2
:1056A000BD018A819B81AC81BD81D5D58A839B83D5
:1056B000AC83BD83A9EAB02D9A8182D9A8EAB02D26
:1056C0009B817ED9A0919502B0919602AA83BB835B
:1056D0000C820D828A819B81AC81BD8149E6502D6F
:1056E000602D702D81D544E6502D602D702DB3D5E1
:1056F0008A839B83AC83BD838A819B81AC81BD817E
:10570000B92FA82F992788278A839B83AC83BD83D1
:10571000E8E5F4E080819181A281B38148EE53E015
:10572000602D702D98D5AC01BD018A819B81AC8123
:10573000BD8191D58A839B83AC83BD83ABEAB02DB9
:105740009A813ED9AAEAB02D9B813AD9A0919502BF
:10575000B0919602AA83BB830C820D828A819B81C1
:10576000AC81BD814FE5502D602D702D3DD544E6B7
:10577000502D602D702D6FD58A839B83AC83BD83A4
:105780008A819B81AC81BD81B92FA82F9927882759
:105790008A839B83AC83BD83E8E5F4E080819181BB
:1057A000A281B38148EE53E0602D702D54D5AC0139
:1057B000BD018A819B81AC81BD814DD58A839B834C
:1057C000AC83BD83ADEAB02D9A81FAD8ACEAB02D96
:1057D0009B81F6D8A5EAB02D98E5F2D8A0EAB02DC5
:1057E00090EEEED8A1EAB02D90ECEAD8B0915C042E
:1057F000B13208F068C0A0919502B0919602A93824
:10580000F3E1BF07E8F4A9E8B02D902DD9D8A1E9BC
:10581000B02D9FE0D5D8A2E9B02D9FEFD1D8A3E954
:10582000B02D90EFCDD8A4E9B02D902DC9D8A9E81E
:10583000B02D94E4C5D8AFE9B02D98E6C1D8C0C06A
:10584000E3E7FAE0A591B5918D01202D302D312FA0
:10585000202F11270027E8E5F4E080819181A281C3
:10586000B38148EE53E0602D702DF5D4AC01BD013D
:10587000D901C801F0D48C019D0108831983A9E8DE
:10588000B02D902D9DD8A1E9B02D998199D8A2E98C
:10589000B02D988195D8A881B9818FEF9FEF9BD4C7
:1058A000A883B983A3E9B02D99818AD8A4E9B02D42
:1058B000988186D8A9E8B02D94EC82D8AFE9B02DB4
:1058C00098E67ED87DC0A0919502B0919602A93845
:1058D000F3E1BF0728F4AFE9B02D98E671D804C012
:1058E000AFE9B02D94E46CD8A9E8B02D902D68D81C
:1058F000B0919A02FB2FF53119F0F83119F122C05D
:10590000E3E7FAE0A591B591A85ABD4F8D01202D8E
:10591000302D312F202F11270027E8E5F4E080817A
:105920009181A281B38148EE53E0602D702D93D414
:10593000AC01BD01D901C8018ED48C019D01088341
:10594000198323C0E3E7FAE0A591B591B695A79531
:10595000A85ABD4F8D01202D302D312F202F11271A
:105960000027E8E5F4E080819181A281B38148EECF
:1059700053E0602D702D6FD4AC01BD01D901C80179
:105980006AD48C019D0108831983A1E9B02D998106
:1059900017D8A2E9B02D988113D8A881B9818FEFCB
:1059A0009FEF19D4A883B983A3E9B02D998108D8B2
:1059B000A4E9B02D988104D8A9E8B02D96E400D8C8
:1059C000A5E9B02D902D0E94E024A6E9B02D902DE0
:1059D0000E94E024B0915C04B032C0F0A8EBB02D7E
:1059E00091E40E94E024AEE0B1E091E40E94E02462
:1059F000B0919902B23051F0ADE1B1E092E80E946D
:105A0000E024A8E2B1E09AE00E94E024A5EAB02DEB
:105A1000902D0E94E024A0EAB02D90EE0E94E02498
:105A2000A1EAB02D90EC0E94E024A6E7B02D0E94E0
:105A30000325FB2EA6E7B02D9F2D977E0E94E02424
:105A4000A7E7B02D0E940325FB2EA7E7B02D9F2DC1
:105A50009F7B0E94E024AEE9B02D98E80E94E024EC
:105A6000B0915C04B032D8F1A0919502B091960249
:105A7000A03DF7E0BF07A8F4B0915C04B13230F468
:105A8000ACE8B02D99E30E94E02405C0ACE8B02D4D
:105A900099E80E94E024ADE8B02D90E40E94E02453
:105AA00031C0A0919502B0919602A031F7E2BF07F4
:105AB00058F4ACE8B02D9CE40E94E024ADE8B02D91
:105AC00090E20E94E0241EC0ACE8B02D9BE40E944E
:105AD000E024ADE8B02D90E20E94E02413C0A09134
:105AE0009502B0919602A031F7E2BF0730F4ACE81E
:105AF000B02D9FEE0E94E02405C0ACE8B02D9DEED5
:105B00000E94E024B0919902B23081F4B0915C041B
:105B1000B13230F4A9EDB02D96E20E94E0240BC022
:105B2000A9EDB02D96E60E94E02405C0A9EDB02DA8
:105B300092E20E94E024B0919A02FB2FF53119F015
:105B4000F83139F006C0A8E7B02D95E10E94E024B5
:105B500005C0A8E7B02D98E10E94E024A5E7B02D8C
:105B60000E940325FB2EF7FE06C0A5E7B02D9F2D52
:105B70009F770E94E0242696F99009911991299126
:105B8000399108953A932A931A93A9E3B02D0E946C
:105B900003253B2FB0919902B13039F4A9E3B02D20
:105BA000932F9D7F0E94E02406C0A9E3B02D932F80
:105BB00092600E94E024B0915C04B03308F441C0CC
:105BC000A0919502B0919602A839FAE3BF0758F068
:105BD000AAE8B02D9BE20E94E024ABE8B02D9AE148
:105BE0000E94E02438C0A0919502B0919602A83599
:105BF000FBE1BF0798F0A0919502B0919602A839F9
:105C0000FAE3BF0758F4AAE8B02D9CE00E94E02414
:105C1000ABE8B02D9BE10E94E0241DC0A09195024D
:105C2000B0919602A835FBE1BF07A8F4AAE8B02D11
:105C30009CE20E94E024ABE8B02D9CE10E94E024AD
:105C40000AC0AAE8B02D9AE10E94E024ABE8B02D8A
:105C500099E00E94E024B0919902FB2FF13031F0DD
:105C6000F23009F44EC0F33009F0C2C0A6E7B02DFF
:105C70000E9403252B2FB22FBF73B0642B2FA6E7F2
:105C8000B02D922F0E94E024A9EDB02D92E20E9447
:105C9000E024AFE1B1E096E90E94E024A0E2B1E0A7
:105CA00094E60E94E024A1E2B1E096E30E94E024A1
:105CB000A2E2B1E093E20E94E024A3E2B1E09EE11F
:105CC0000E94E024A4E2B1E099E10E94E024B091B6
:105CD0009902B13031F4AEE1B1E0902D0E94E024A0
:105CE00005C0AEE1B1E090E80E94E024A7E2B1E097
:105CF000E0919802FF27EE59F54F94910E94E0241D
:105D000077C0A6E7B02D0E9403251B2FB12FBF73CC
:105D1000B0681B2FA6E7B02D912F0E94E024AAE8BF
:105D2000B02D9AE10E94E024ABE8B02D99E00E94EA
:105D3000E024B0915C04B13230F4A9EDB02D96E2CC
:105D40000E94E02405C0A9EDB02D96E60E94E02453
:105D5000A7EEB02D9FEF0E94E024A8EEB02D90EFAB
:105D60000E94E024A9EEB02D902D0E94E024AAEE1E
:105D7000B02D902D0E94E024ABEEB02D902D0E940E
:105D8000E024ACEEB02D902D0E94E024ADEEB02DBD
:105D9000902D0E94E024AEEEB02D902D0E94E024C4
:105DA000AFEEB02D902D0E94E024A0EFB02D902DED
:105DB0000E94E024A1EFB02D902D0E94E024A2EFDC
:105DC000B02D902D0E94E024A3EFB02D902D0E94C5
:105DD000E024A4EFB02D902D0E94E024A5EFB02D7B
:105DE000902D0E94E024A6EFB02D9FE00E94E024B9
:105DF000A5E7B02D0E9403253B2F37FF06C0A5E77E
:105E0000B02D932F9F770E94E0240E9415261991B0
:105E10002991399108953A932A931A930A93FA9201
:105E2000B0919902FB2FF13029F0F230A9F1F33053
:105E300009F001C1A2E7B02D0E9403250B2FA2E7B4
:105E4000B02D902F94600E94E024B0915C04B03398
:105E5000E8F0A5E2B1E00E940325BF710B2F0D30E1
:105E600059F4A7EFB02D98E90E94E024A8EFB02DD7
:105E700098E10E94E0240AC0A7EFB02D98E10E94AB
:105E8000E024A8EFB02D98E10E94E024A3E7B1E060
:105E900095E70E94E024CFC0AAE8B02D902D0E9483
:105EA000E024ABE8B02D902D0E94E024A3E7B02DB4
:105EB0000E9403250B2FA02FBB27AC77B02DB695E2
:105EC000A795B695A7952A2FB02FB170FB2E2C3031
:105ED00010F4302D0CC0223118F4B1E03B2F07C074
:105EE000283118F4B2E03B2F02C0B3E03B2F01FD94
:105EF00034C0B22FAF2D0E94C5261B2F2C3030F49A
:105F0000AEEDB02D912F0E94E0240CC0223150F450
:105F1000AEEDB02D9AE20E94E024AFEDB02D912FAE
:105F20000E94E024223108F45AC0283158F4AEED22
:105F3000B02D9AE20E94E024A0EEB02D912F0E9495
:105F4000E0244DC0AEEDB02D9AE20E94E024A1EE17
:105F5000B02D912F0E94E02442C0283118F4B2E005
:105F60003B2F0BC0223118F4B1E03B2F06C02C3080
:105F700010F4302D02C0B3E03B2FB32F0E94362621
:105F80001B2F301531F4AEEDB02D912F0E94E0247F
:105F900026C0313059F4AEEDB02D9AE20E94E024D3
:105FA000AFEDB02D912F0E94E02419C0323059F48A
:105FB000AEEDB02D9AE20E94E024A0EEB02D912F1C
:105FC0000E94E0240CC0333051F4AEEDB02D9AE2C3
:105FD0000E94E024A1EEB02D912F0E94E024A8E7BA
:105FE000B02D9FE10E94E024A8E7B02D9CE10E9423
:105FF000E024B0915C04B13230F4A9EDB02D96E20A
:106000000E94E02405C0A9EDB02D96E60E94E02490
:10601000B0919A02FB2FF53119F0F83139F006C032
:10602000A8E7B02D95E10E94E02405C0A8E7B02DB7
:1060300098E10E94E024F9900991199129913991F0
:1060400008953A933B2FA4E7B02D0E940325B32374
:10605000AB2FBB27832F9927A817B90711F4B1E0FD
:1060600001C0B02D39910895B1FF02C0B1E008958B
:10607000B02D0895089500002298B4B1BB60B4B962
:106080002998B5B1BD60B5B90895009213022B9857
:1060900001C0000083B182FB882780F98130C9F3F9
:1060A0002CC080911202815080931202E091120262
:1060B000FF27E85CFC4FA081B02D902DBB0FA7FD02
:1060C00002C0289804C085B18E7F8F5F85B9299A58
:1060D00083B182FB882780F9B80F2998AA0F9F5FA8
:1060E000983060F3E0911302FF27E852FD4FB08330
:1060F000809113028F5F80931302809112028015AA
:1061000081F62B9A00000895B02DB02DA0E2EB2F60
:10611000FF27E852FD4FA083BF5FB036B8F300926F
:1061200013020895B02DB02DA0E2EB2FFF27E85CFD
:10613000FC4FA083BF5FB036B8F3009212020895FF
:106140003A93E2DFEFDFBFE23B2FE32FFF27E75A6F
:10615000FD4FB081EFE2FF27932FAA27E91BFA0B2F
:10616000E85CFC4FB0833150301579F7B0E4B09360
:106170006703B0E3B093120288DF399108953A9330
:106180002B98302D00003F5F3E3FE0F32B9A302DDF
:1061900000003F5F3F34E0F32B98B0E3B093380347
:1061A000B1E0B093120271DF399108950C949FDC35
:1061B000EB2FE92799231CF4909581959F4FBB23E2
:1061C0001CF4B095A195BF4F33D0EE231CF4B095CD
:1061D000A195BF4F08958A9FB0019A9F700DB89FF7
:1061E000700DDB01002408953A932A93489FF00133
:1061F0004A9F9001499FF00D211D0024301D589F9A
:10620000F00D211D0024301D599F200D311D689F68
:10621000200D311D4B9F300D5A9F300D699F300D61
:10622000789F300DD901CF0100242991399108952B
:1062300077276627F0E1AA0FBB1F661F771F681735
:10624000790718F0681B790BA395FA95A1F70895C3
:10625000EFDFDB01089568943A932A931A930A9327
:106260003327222711270027F0E2880F991FAA1F42
:10627000BB1F001F111F221F331F041715072607FE
:10628000370728F0041B150B260B370B8395FA955F
:1062900061F716F0D901C801099119912991399135
:1062A0000895FD019D919923E9F7AE1BBF0B11974E
:1062B00008953A932A931A930A93FA92EA92DA92F9
:1062C000CA9228977D016C01A8E0BB278D01DE01F1
:1062D00050969D01EC82FD820E820F82AFEFBFE7E8
:1062E000AA83BB83DE01C601B9018DD02896C9906F
:1062F000D990E990F99009911991299139910895CE
:106300003A932A931A930A93FA929D01192FF9014D
:10631000A481B5811097F1F0F901A081B1811196A6
:10632000F90182819381A817B90709F4102DF901A9
:10633000A081B181F90182819381A817B90750F436
:10634000F901A081B181F90184819581A80FB91F5C
:10635000FD011083F901A681B7811097A1F0F90121
:10636000A081B181F90182819381A817B90758F4FE
:10637000F901A681B781FA2E0B2FA12FBB27C901E6
:10638000F02FEF2D0995F901A081B1811196A0831D
:10639000B183F990099119912991399108953A930E
:1063A0002A931A930A93FA92EA929D018C017B0137
:1063B00003C0D701922FA4DF015010091030CCF791
:1063C000E990F990099119912991399108953A9399
:1063D0002A931A930A93FA92EA929D018C017B0107
:1063E00024FD0AC031FD03C0A0E2B02D02C0A0E32D
:1063F000B02DC801B701D3DFE990F9900991199147
:106400002991399108953A932A931A930A93FA920B
:10641000EA92DA92CA92BA92AA929A928A927A925C
:106420006A925A924A923A926097DA2EEB2E8E83B3
:106430009F8368877987ED2DFE2D00820182D7C268
:10644000F5E2FF1629F0BE2DAD2D9F2D59DFCFC2ED
:10645000B02CC02C702C802C202D302D502C602C7A
:10646000EE81FF81DF013196EE83FF83FD01B08174
:10647000FB2EFB2FF03259F0F33259F0F73259F07E
:10648000FB3259F0FD3259F0F03359F00DC0206461
:10649000E7CF2068E5CF3068E3CF2062E1CF20610D
:1064A000DFCF3260DDCF00C0FAE2FF1699F5E88554
:1064B000F9853296E887F9873297A081B181BA2EA3
:1064C000CB2EF0E0CF1644F4BC2DAB2DB095A195AA
:1064D000BF4FBA2ECB2E2061EE81FF81DF013196B6
:1064E000EE83FF83FD01B081FB2E1CC013C0BC2DC9
:1064F000AB2D8AE0902D6FDEAF0DB01DD097BA2E78
:10650000CB2EEE81FF81DF013196EE83FF83FD010B
:10651000B081FB2EAF2DBB27A033B0051CF0FAE3F2
:10652000FF1628F3F0E0CF1614F4B02CC02CFEE2D6
:10653000FF1609F040C0EE81FF81DF013196EE8346
:10654000FF83FD01B081FB2EFAE2FF1641F5E885DD
:10655000F9853296E887F9873297A081B1817A2E42
:106560008B2EEE81FF81DF013196EE83FF83FD01EB
:10657000B081FB2E1CC013C0B82DA72D8AE0902D32
:106580002ADEAF0DB01DD0977A2E8B2EEE81FF81C3
:10659000DF013196EE83FF83FD01B081FB2EAF2D2D
:1065A000BB27A033B0051CF0FAE3FF1628F3F0E098
:1065B0008F160CF03160F8E6FF16B9F4EE81FF811A
:1065C000DF013196EE83FF83FD01B081FB2EB836EB
:1065D00059F42860EE81FF81DF013196EE83FF835D
:1065E000FD01B081FB2E01C02460FF2DF03009F4C5
:1065F00041C0F53209F441C0F83509F4C8C0F3369A
:1066000009F440C0F43609F4E1C0F93609F4DEC0FB
:10661000FE3609F456C0FF3609F4CAC0F03709F453
:10662000A1C0F33709F471C0F53709F4CBC0F837CE
:1066300009F4AEC000C0A0915D04B0915E04109753
:1066400009F4D5C1A0915D04B0915E043A2E4B2EA1
:10665000DE011896BA93AA938A927A92BF2DAE2D34
:106660009D2D832F722F6C2D5B2DF42DE32D09951D
:106670002496BDC1AFEFBFEFE7C1BE2DAD2D9F2D5D
:106680003FDED5C0E885F9853296E887F9873297ED
:10669000B081FB2EF1E0BF1AC008D9019C2D8B2DD3
:1066A0007E2D6D2D94DEBE2DAD2D9F2D29DE24FF78
:1066B00007C0A0E2B02D9C2D8B2D7E2D6D2D6FDEA1
:1066C00096C123FF0FC0FE2DED2DB081E885F98521
:1066D0003296E887F98732979081A181E92FFA2FC6
:1066E000B08385C1E885F9853296E887F9873297C6
:1066F000A081B181AC83BD83FE2DED2DA081B18140
:10670000EC81FD81A083B18372C1E885F985329661
:10671000E887F9873297A081B1818D01D801C1DD69
:106720009A2EAB2E30FF05C079148A0414F4A82CDD
:10673000972CB918CA08D9019C2D8B2D7E2D6D2D53
:1067400046DE08C0BE2DAD2DC8010F5F1F4FFC01F6
:106750009081D6DDBA2DA92DF1E09F1AA0081097DF
:1067600089F7A5CFE885F9853296E887F9873297CA
:10677000A081B1818D0127FF04C0A3E2BB275A2E5F
:106780006B2E3160A4E0BB277A2E8B2E50C0306276
:1067900027FF0AC0F8E7FF1619F0A8E5B0E302C02A
:1067A000A8E7B0E35A2E6B2E30FF01C03D7F0FC02B
:1067B00027FF04C0A0E3BB275A2E6B2E30FF01C079
:1067C0003D7F05C030FF01C03D7F01C03064E885DA
:1067D000F9853296E887F9873297A081B1818D01DA
:1067E00036FF1EC023FF02C0102D00C0103054F42D
:1067F000AA27BB27A01BB10B8D01ADE2BB275A2EE8
:106800006B2E11C025FF05C0ABE2BB275A2E6B2EA5
:106810000AC026FF04C0A0E2BB275A2E6B2E03C07D
:1068200023FF01C0102D30FF01C03D7F00C0902C20
:10683000A02C30FD04C0A1E0BB277A2E8B2EFF2DAB
:10684000F835A1F1F43609F476C0F93609F473C0CD
:10685000FF3609F442C0F03749F1F53709F46BC04F
:10686000F83721F16CC022C035FF0CC0F801EF7081
:10687000F02DE458F54FB491FE013A96E90DFA1D5A
:10688000B0830BC0F801EF70F02DE457F54FB491D1
:10689000FE013A96E90DFA1DB083FFEF9F1AFFEF54
:1068A000AF0AB4E016950795BA95E1F70015100503
:1068B000D9F645C012C0B02FB770B05DFE013A9650
:1068C000E90DFA1DB083FFEF9F1AFFEFAF0A16958F
:1068D000079516950795169507950015100559F714
:1068E0002EC029C0D901A02DB078109789F0BA2DFB
:1068F000A92DA370B02DA330B00551F4BCE2FE0168
:106900003A96E90DFA1DB083FFEF9F1AFFEFAF0A29
:10691000D8018AE0902D9CDCA05DFE013A96E90D3D
:10692000FA1DA083FFEF9F1AFFEFAF0AD8018AE09C
:10693000902D7EDC8D0100151005A1F600C07918A0
:106940008A08F0E08F1614F4702C802CB718C80851
:10695000B918CA08F1E06F1618F0F1E0BF1AC008C4
:106960005014600419F0F1E0BF1AC00831FD08C0EE
:10697000D9019C2D8B2D7E2D6D2D29DDB02CC02CA9
:10698000F1E06F1640F0BE2DAD2D962D852D892F8F
:106990009927982FB5DC5014600421F0BE2DAD2D41
:1069A000952DAEDCD9019C2D8B2D7E2D6D2D0FDD0F
:1069B000A0E3B02D982D872D7E2D6D2DF0DC08C025
:1069C000BE2DAD2DFE013A96E90DFA1D908198DCA1
:1069D000F1E09F1AA008F0E0AF1694F724FF07C07B
:1069E000A0E2B02D9C2D8B2D7E2D6D2DD8DCEE815F
:1069F000FF81DF013196EE83FF83FD01B081FB2E25
:106A0000B01509F01DCDFE2DED2DA481B581109797
:106A1000B9F0FE2DED2DA081B181FE2DED2D8281ED
:106A20009381A817B90760F4FE2DED2DA081B181E7
:106A3000FE2DED2D84819581A80FB91FFD010082E7
:106A4000FE2DED2DA081B18160963990499059902D
:106A50006990799089909990A990B990C990D990AE
:106A6000E990F990099119912991399108950000BF
:106A70000000000000000000000000000000000016
:106A80000000000000000000000000000000000006
:106A900000000000000000000000000000000000F6
:106AA00000000000000000000000000000000000E6
:10F0100016266829B42D5642FFFFFFFFFFFFFFFFB2
:10F02000DB2D566C6B03010001DB2D566C6B03016D
:10F030000001FF4153545241203139130026FFFF94
:10F04000B22E486C6B022000019E2E566C6B022083
:10F050000001FF41535452412032381C0023FFFF6E
:10F06000F62D566C6B023E0101F62D566C6B023E7E
:10F070000101FF484F5442495244200D0026FFFF32
:10F08000DB2D566C6B05030002DB2D566C6B050304
:10F090000002FF4153545241203233170026FFFF34
:10F0A000472D56204E02FA2001472D56204E02FAD7
:10F0B0002001FF41544C4249524433FBFF26FFFFDD
:10F0C000042B56307503010002042B5630750301E2
:10F0D0000002FF48454C4C41532032270026FFFFD9
:10F0E0008E2D486C6B022000018E2D486C6B022027
:10F0F0000001FF45554249524420311C0023FFFFC7
:10F10000F62D486C6B03550001F62D486C6B0355CA
:10F110000001FF4153545241203545050026FFFFB1
:10F12000823056606D07460001823056606D07469A
:10F130000001FF54484F5220202020FFFF26FFFFF0
:10F14000432E566C6B039E0001432E566C6B039E40
:10F150000001FF4555524249524439090026FFFF3C
:10F16000FFFFFFFFFFFFFFFFFFFFFFFFFFFFFFFFAF
:10F17000FFFFFFFFFFFFFFFFFFFFFFFFFFFFFFFF9F
:10F18000FFFFFFFFFFFFFFFFFFFFFFFFFFFFFFFF8F
:10F19000FFFFFFFFFFFFFFFFFFFFFFFFFFFFFFFF7F
:10FDE0000700FFFFFFFFFFFFFFFFFFFFFFFFFFFF1A
:10FDF00055FF0AFFFFFFFFFFFFFFFFFFFFFFFFFFB2
:10FE0000FFFFFFFFFFFF6204FFFF4104FFFF6D04E0
:10FE1000FFFF4C04FFFF7804FFFF1504FFFF4104C0
:10FE2000FFFF7804FFFF7804FFFF6D04FFFFFFFF73
:10FE3000FFFFFFFFFFFFFFFFFFFFFFFFFFFFFFFFD2
:10FE4000FFFFFFFFFFFFFFFFFFFFFFFFFFFFFFFFC2
:10FE5000FFFFFFFFFFFFFFFFFFFFFFFFFFFFFFFFB2
:10FE6000FFFFFFFFFFFFFFFFFFFFFFFFFFFFFFFFA2
:10FE7000FFFFFFFFFFFFFFFFFFFFFFFFFFFFFFFF92
:10FE8000FFFFFFFFFFFFFFFFFFFFFFFFFFFFFFFF82
:10FE9000FFFFFFFFFFFFFFFFFFFFFFFFFFFFFFFF72
:10FEA000FFFFFFFFFFFFFFFFFFFFFFFFFFFFFFFF62
:10FEB000FFFFFFFFFFFFFFFFFFFFFFFFFFFFFFFF52
:10FEC000FFFFFFFFFFFFFFFFFFFFFFFFFFFFFFFF42
:10FED000FFFFFFFFFFFFFFFFFFFFFFFFFFFFFFFF32
:10FEE000FFFFFFFFFFFFFFFFFFFFFFFFFFFFFFFF22
:10FEF000FFFFFFFFFFFFFFFFFFFFFFFFFFFFFFFF12
:10FF0000FFFFFFFFFFFFFFFFFFFFFFFFFFFFFFFF01
:10FF1000FFFFFFFFFFFFFFFFFFFFFFFFFFFFFFFFF1
:10FF2000FFFFFFFFFFFFFFFFFFFFFFFFFFFFFFFFE1
:10FF3000FFFFFFFFFFFFFFFFFFFFFFFFFFFFFFFFD1
:10FF4000FFFFFFFFFFFFFFFFFFFFFFFFFFFFFFFFC1
:10FF5000FFFFFFFFFFFFFFFFFFFFFFFFFFFFFFFFB1
:10FF6000FFFFFFFFFFFFFFFFFFFFFFFFFFFFFFFFA1
:10FF7000FFFFFFFFFFFFFFFFFFFFFFFFFFFFFFFF91
:10FF8000FFFFFFFFFFFFFFFFFFFFFFFFFFFFFFFF81
:10FF9000FFFFFFFFFFFFFFFFFFFFFFFFFFFFFFFF71
:10FFA000FFFFFFFFFFFFFFFFFFFFFFFFFFFFFFFF61
:10FFB000FFFFFFFFFFFFFFFFFFFFFFFFFFFFFFFF51
:10FFC000FFFFFFFFFFFFFFFFFFFFFFFFFFFFFFFF41
:10FFD000FFFFFFFFFFFFFFFFFFFFFFFFFFFFFFFF31
:10FFE000FFFFFFFFFFFFFFFFFFFFFFFFFFFFFFFF21
:10FFF000FFFFFFFFFFFFFFFFFFFFFFFF3D29ED5565
:00000001FF
